:1000000000800010CD00000061190000631900009D
:100010006519000067190000691900000000000060
:100020000000000000000000000000006B1900004C
:100030006D190000000000006F1900007119000028
:100040007319000073190000731900007319000080
:100050007319000073190000731900007319000070
:100060007319000073190000731900007319000060
:100070007319000073190000731900007319000050
:100080007319000073190000AD040000731900001B
:100090007319000073190000731900007319000030
:1000A0007319000073190000731900007319000020
:1000B000E5010000731900007319000073190000B6
:1000C000731900007319000073190000014880477C
:1000D000014800474154000005AF000040F238538A
:1000E000C1F200031A780AB901201870704700BFE6
:1000F00040F20000C1F2000008B503682BB140F2E5
:100100000003C0F2000303B1984708BD84B001901A
:10011000019B03F0070303934EF60053CEF2000356
:10012000DB680293029A4FF6FF03C0F2000302EA73
:1001300003030293039B4FEA0322029B42EA030359
:1001400043F0BE6343F4202302934EF60053CEF2F5
:100150000003029ADA6004B0704700BF82B0034621
:100160008DF807304EF20013CEF200039DF9072000
:100170004FEA52129DF8071001F01F014FF00100E5
:1001800000FA01F143F8221002B0704782B0034632
:1001900000918DF807309DF90730002B11DA4EF6EB
:1001A0000053CEF200039DF8072002F00F02A2F1E7
:1001B0000401009AD2B24FEAC202D2B20B441A76BC
:1001C0000DE04EF20013CEF200039DF90710009AE5
:1001D000D2B24FEAC202D2B20B4483F8002302B07B
:1001E000704700BF00B585B04FE14FF0A043039AC0
:1001F000C3F8E82F039B03F00103DBB2002B19D0F7
:1002000040F23C53C1F200031B6803F1010240F2CB
:100210003C53C1F200031A6043F2A413C1F200037D
:100220001B684CF20000C4F200004AF66471C0F290
:1002300000019847039B03F00203002B20D04FF0EE
:10024000806002F051FD0346002B19D140F240536B
:10025000C1F200031B6803F1010240F24053C1F2F6
:1002600000031A6043F2A413C1F200031B684CF2AE
:100270000000C4F200004AF67071C0F20001984715
:10028000039B03F00403002B19D040F24C53C1F23E
:1002900000031B6803F1010240F24C53C1F200035A
:1002A0001A6043F2A413C1F200031B684CF2000071
:1002B000C4F200004AF67C71C0F200019847039B2B
:1002C00003F00803002B53D002F0E4FC0346002B9C
:1002D00034D04FF0804002F007FD0346002B2AD0B7
:1002E00002F01AFD0346A3F103030293029B762B4F
:1002F00022D840F20000C1F6903002F0F5FC03462F
:10030000002B19D140F25C53C1F20003029A1A602B
:1003100043F24403C1F200030193029B00936B4636
:10032000184602F047FC40F26053C1F200034FF060
:1003300001021A7000E000BF02F002FD43F2A413B4
:10034000C1F200031B684CF20000C4F200004AF640
:100350008871C0F20001984740F25853C1F200037F
:100360001B6803F1010240F25853C1F200031A6006
:10037000039B03F01003002B19D040F24453C1F249
:1003800000031B6803F1010240F24453C1F2000371
:100390001A6043F2A413C1F200031B684CF2000080
:1003A000C4F200004AF69071C0F200019847039B26
:1003B00003F02003002B19D040F24853C1F2000390
:1003C0001B6803F1010240F24853C1F200031A60B6
:1003D00043F2A413C1F200031B684CF20000C4F204
:1003E00000004AF6A071C0F200019847039B03F099
:1003F0004003002B19D040F25053C1F200031B6898
:1004000003F1010240F25053C1F200031A6043F2BB
:10041000A413C1F200031B684CF20000C4F20000F8
:100420004AF6AC71C0F200019847039B03F08003C9
:10043000002B19D040F25453C1F200031B6803F1A2
:10044000010240F25453C1F200031A6043F2A413B4
:10045000C1F200031B684CF20000C4F200004AF62F
:10046000B871C0F200019847039B03F40053002BBE
:100470000BD040F26453C1F200031B6803F1010288
:1004800040F26453C1F200031A604FF0A043D3F866
:10049000E02F4FF0A043D3F8E43F02EA03030393B5
:1004A000039B002B7FF4A1AE05B000BD4CF200030E
:1004B000C4F20F034CF20002C4F20F02D2F8402142
:1004C00042F00102C3F8402140F26153C1F200033F
:1004D0004FF001021A70704700B587B001904FF0DD
:1004E00064030593019B4FF000021A70019B03F116
:1004F00001034FF050021A70019B03F102036FF0E9
:1005000025021A70019B03F103034FF06B021A706E
:10051000019B03F104036FF079021A70019B03F150
:1005200005036FF01C021A70019B03F106034FF0E4
:100530000C021A70019B03F107034FF01D021A70A1
:10054000019B03F108034FF012021A70019B03F1A3
:1005500009036FF01F021A70019B03F10A034FF0A9
:100560001F021A70019B03F10B034FF010021A7067
:10057000019B03F10C03059AD2B21A70019B03F19F
:100580000D03059A4FEA1222D2B21A704FF00003FF
:1005900003930BE0039B03F10E02019B13444FF006
:1005A00055021A70039B03F101030393039A059B01
:1005B0009A42EFD301984FF0720100F053FB0346CB
:1005C0000493019B03F17203049AD2B21A70019B47
:1005D00003F17303049A4FEA1222D2B21A70019BFC
:1005E00003F17403049A4FEA1242D2B21A70019BCB
:1005F00003F17503049A4FEA1262D2B21A7007B07F
:1006000000BD00BF00B583B04FF000038DF802308D
:100610004FF000038DF804304FF000038DF80330E5
:100620004FF001038DF800304FF012038DF80130C8
:100630006B46184603F06EF94FF000038DF8023058
:100640004FF000038DF804304FF000038DF80330B5
:100650004FF003038DF800304FF01A038DF801308E
:100660006B46184603F056F94FF003004FF08061D7
:100670004FF0010202F042FC4FF001004FF48021E4
:100680004FF0010202F03AFC4FF003004FF080619E
:1006900002F05EFC4FF001004FF4802102F058FCA4
:1006A00003B000BD00B585B00190019B012B14BFC4
:1006B00000230123DAB2019B032B14BF0023012383
:1006C000DBB242EA0303DBB2002B05D04FF001009E
:1006D0004FF4802102F052FC019B022B14BF002337
:1006E0000123DAB2019B032B14BF00230123DBB2E9
:1006F00042EA0303DBB2002B05D04FF003004FF0BA
:10070000806102F03BFC4FF00003039303E0039B86
:1007100003F101030393039A4FF6FF73C0F20F0333
:100720009A42F4D9019B012B14BF00230123DAB2B2
:10073000019B032B14BF00230123DBB242EA030316
:10074000DBB2002B05D04FF001004FF4802102F006
:10075000FFFB019B022B14BF00230123DAB2019B94
:10076000032B14BF00230123DBB242EA0303DBB2F5
:10077000002B05D04FF003004FF0806102F0E8FB42
:100780004FF00003039303E0039B03F10103039382
:10079000039A4FF6FF73C0F20F039A42F4D905B0E3
:1007A00000BD00BF00B583B04FF001038DF80230EB
:1007B0004FF000038DF804304FF000038DF8033044
:1007C0004FF00A038DF801304FF002038DF800302E
:1007D0006B46184603F09EF84CF20003C4F20F0378
:1007E0004FF00002C3F840214CF20003C4F20F03A3
:1007F0004FF00002C3F848214CF20003C4F20F038B
:100800004FF00002C3F84C214CF20003C4F20F0376
:100810004FF00F02C3F848214CF20003C4F20F035B
:100820004FF00002C3F84C214CF20003C4F20F0356
:100830004FF00F02C3F840214FF012004FF00401B7
:10084000FFF7A4FC4FF01200FFF788FC03B000BDD7
:1008500000B58BB04FF001038DF816304FF0000358
:100860008DF818304FF000038DF817304FF001036A
:100870008DF814304FF000038DF8153005AB184695
:1008800003F048F84FF001038DF8153005AB18461A
:1008900003F040F84FF004038DF8153005AB18460F
:1008A00003F038F84FF008038DF8153005AB184603
:1008B00003F030F84FF009038DF8153005AB1846FA
:1008C00003F028F84FF00A038DF8153005AB1846F1
:1008D00003F020F84FF00E038DF8153005AB1846E5
:1008E00003F018F84FF00F038DF8153005AB1846DC
:1008F00003F010F84FF010038DF8153005AB1846D3
:1009000003F008F84FF011038DF8153005AB1846C9
:1009100003F000F843F2A413C1F200031B684CF289
:100920000000C4F200004AF6C071C0F2000198470E
:1009300040F20803C1F200031B781A4640F2080394
:10094000C1F200035B789C4640F20803C1F2000349
:100950009B789E4640F20803C1F20003DB781846FC
:1009600040F20803C1F200031B79194640F2080364
:10097000C1F200035B79CDF800E00190029103938E
:1009800043F24C10C1F200004AF6D471C0F20001EB
:10099000634605F0DBFC43F29C13C1F200031B68C5
:1009A0004CF20000C4F2000043F24C11C1F200010D
:1009B00098474FF00003079340F20803C1F2000389
:1009C000089318E043F2A413C1F200031B684CF231
:1009D0000000C4F200004AF6FC71C0F20001984722
:1009E0004FF48013099303E0099B03F1FF3309934C
:1009F000099B002BF8D107AB184601F0F7FD034621
:100A0000002BDFD04FF0FF004FF0010102F006F99C
:100A10004FF01C004FF00001FFF7B8FB4FF01C0037
:100A2000FFF79CFB43F2A413C1F200031B684CF2D6
:100A30000000C4F200004BF23401C0F200019847FC
:100A40000BB000BD00B589B04FF0000306934BF228
:100A50008C02C0F2000201AB92E80300186003F1BF
:100A6000040319804FF00400FFF750FBFFF7CAFDA5
:100A700001F03EFBFFF7ECFEFFF794FE43F2C803E4
:100A8000C1F2000305930598FFF726FD01AB184658
:100A90004FF0010101F0C2FF43F2A413C1F20003C1
:100AA0001B684CF20000C4F200004BF25001C0F28F
:100AB000000198474FF440504FF0010102F000F858
:100AC0004FF00003069307E04FF00100FFF7EAFD47
:100AD000069B03F101030693069B042BF4D972B61F
:100AE0004CF20003C4F20F034FF00002C3F8C02021
:100AF00030BF04F0A5FC01F0FBFAFFF783FD43F2E1
:100B0000A413C1F200031B684CF20000C4F2000001
:100B10004BF26801C0F200019847FFF799FE62B6F8
:100B200003E04FF00300FFF7BDFD40F26153C1F257
:100B300000031B78DBB2002BF3D040F26153C1F20B
:100B400000034FF000021A7043F2C803C1F2000321
:100B5000059343F2A413C1F200031B684CF200009A
:100B6000C4F200004BF28001C0F2000198474FF040
:100B70000200FFF797FD059B04934FF07603039364
:100B800003AB184601F0D8FF02F0F2F84FF0000373
:100B9000079303E0079B03F101030793079A4FF6BE
:100BA000FF73C0F21F039A42F4D900BFBDE700BF34
:100BB00008B5FFF747FF0346184608BD82B001900D
:100BC0000091FEE782B00190019B4FF0FF321A6066
:100BD00002B0704788B001900B468DF80330019B3E
:100BE0001B68069348F22033CEF6B85304939DF861
:100BF0000320069B82EA030303F0FF0305934FF0F3
:100C00000003039315E0059B03F00103DBB2002B07
:100C100007D0059B4FEA5302049B82EA0303059326
:100C200003E0059B4FEA53030593039B03F1010384
:100C30000393039B072BE6D9069B4FEA1322059BE0
:100C400082EA03030793019B079A1A6008B0704772
:100C500082B00190019B1B686FEA0302019B1A603E
:100C600002B0704700B585B00190009102AB184604
:100C7000FFF7A8FF019B03930AE0039B1B7802AADE
:100C800010461946FFF7A6FF039B03F101030393E8
:100C9000009B002B0CBF00230123DBB2009A02F162
:100CA000FF320092002BE8D102AB1846FFF7D0FFCD
:100CB000029B184605B000BD84B00190019B03F073
:100CC000070303934EF60053CEF20003DB68029352
:100CD000029A4FF6FF03C0F2000302EA03030293F5
:100CE000039B4FEA0322029B42EA030343F0BE63E5
:100CF00043F4202302934EF60053CEF20003029AEF
:100D0000DA6004B0704700BF82B003468DF8073048
:100D10004EF20013CEF200039DF907204FEA521263
:100D20009DF8071001F01F014FF0010000FA01F1DA
:100D300043F8221002B0704782B0034600918DF84C
:100D400007309DF90730002B11DA4EF60053CEF232
:100D500000039DF8072002F00F02A2F10401009A9F
:100D6000D2B24FEAC202D2B20B441A760DE04EF272
:100D70000013CEF200039DF90710009AD2B24FEA99
:100D8000C202D2B20B4483F8002302B0704700BF06
:100D900000B585B04FE14FF0A043039AC3F8E82FA8
:100DA000039B03F00103DBB2002B19D040F23C534C
:100DB000C1F200031B6803F1010240F23C53C1F28F
:100DC00000031A6043F2A413C1F200031B684CF243
:100DD0000000C4F200004BF29401C0F200019847F9
:100DE000039B03F00203002B20D04FF0806001F042
:100DF0007BFF0346002B19D140F24053C1F20003A0
:100E00001B6803F1010240F24053C1F200031A6073
:100E100043F2A413C1F200031B684CF20000C4F2B9
:100E200000004BF2A001C0F200019847039B03F0C1
:100E30000403002B19D040F24C53C1F200031B688D
:100E400003F1010240F24C53C1F200031A6043F275
:100E5000A413C1F200031B684CF20000C4F20000AE
:100E60004BF2AC01C0F200019847039B03F008036A
:100E7000002B53D001F00EFF0346002B34D04FF06F
:100E8000804001F031FF0346002B2AD001F044FFDF
:100E90000346A3F103030293029B762B22D840F270
:100EA0000000C1F6903001F01FFF0346002B19D15E
:100EB00040F25C53C1F20003029A1A6043F2440309
:100EC000C1F200030193029B00936B46184601F0A8
:100ED00071FE40F26053C1F200034FF001021A703C
:100EE00000E000BF01F02CFF43F2A413C1F20003A5
:100EF0001B684CF20000C4F200004BF2B801C0F2D3
:100F00000001984740F25853C1F200031B6803F1F7
:100F1000010240F25853C1F200031A60039B03F030
:100F20001003002B19D040F24453C1F200031B6898
:100F300003F1010240F24453C1F200031A6043F28C
:100F4000A413C1F200031B684CF20000C4F20000BD
:100F50004BF2C001C0F200019847039B03F020034D
:100F6000002B19D040F24853C1F200031B6803F173
:100F7000010240F24853C1F200031A6043F2A41385
:100F8000C1F200031B684CF20000C4F200004BF2F7
:100F9000D001C0F200019847039B03F04003002BEF
:100FA00019D040F25053C1F200031B6803F1010253
:100FB00040F25053C1F200031A6043F2A413C1F28D
:100FC00000031B684CF20000C4F200004BF2DC018D
:100FD000C0F200019847039B03F08003002B19D057
:100FE00040F25453C1F200031B6803F1010240F2C6
:100FF0005453C1F200031A6043F2A413C1F2000378
:101000001B684CF20000C4F200004BF2E801C0F291
:1010100000019847039B03F40053002B0BD040F2D0
:101020006453C1F200031B6803F1010240F26453F0
:10103000C1F200031A604FF0A043D3F8E02F4FF045
:10104000A043D3F8E43F02EA03030393039B002B7E
:101050007FF4A1AE05B000BD4CF20003C4F20F0353
:101060004CF20002C4F20F02D2F8402142F0010219
:10107000C3F8402140F26153C1F200034FF0010276
:101080001A70704700B587B001904FF06403059364
:10109000019B4FF000021A70019B03F101034FF016
:1010A00050021A70019B03F102036FF025021A70BF
:1010B000019B03F103034FF06B021A70019B03F1D4
:1010C00004036FF079021A70019B03F105036FF0BE
:1010D0001C021A70019B03F106034FF00C021A70F8
:1010E000019B03F107034FF01D021A70019B03F1EE
:1010F00008034FF012021A70019B03F109036FF00D
:101100001F021A70019B03F10A034FF01F021A70AD
:10111000019B03F10B034FF010021A70019B03F1C6
:101120000C03059AD2B21A70019B03F10D03059AC4
:101130004FEA1222D2B21A704FF0000303930BE071
:10114000039B03F10E02019B13444FF055021A70EA
:10115000039B03F101030393039A059B9A42EFD388
:1011600001984FF07201FFF77DFD03460493019B48
:1011700003F17203049AD2B21A70019B03F1730354
:10118000049A4FEA1222D2B21A70019B03F174033F
:10119000049A4FEA1242D2B21A70019B03F175030E
:1011A000049A4FEA1262D2B21A7007B000BD00BFB3
:1011B00000B583B04FF000038DF802304FF000030C
:1011C0008DF804304FF000038DF803304FF0010329
:1011D0008DF800304FF012038DF801306B46184641
:1011E00002F098FB4FF000038DF802304FF000033F
:1011F0008DF804304FF000038DF803304FF00303F7
:101200008DF800304FF01A038DF801306B46184608
:1012100002F080FB4FF003004FF080614FF00102BD
:1012200001F06CFE4FF001004FF480214FF00102FD
:1012300001F064FE4FF003004FF0806101F088FE82
:101240004FF001004FF4802101F082FE03B000BD99
:1012500000B585B00190019B012B14BF0023012331
:10126000DAB2019B032B14BF00230123DBB242EA55
:101270000303DBB2002B05D04FF001004FF48021B7
:1012800001F07CFE019B022B14BF00230123DAB284
:10129000019B032B14BF00230123DBB242EA0303AB
:1012A000DBB2002B05D04FF003004FF0806101F05E
:1012B00065FE4FF00003039303E0039B03F101037A
:1012C0000393039A4FF6FF73C0F20F039A42F4D9C7
:1012D000019B012B14BF00230123DAB2019B032BD6
:1012E00014BF00230123DBB242EA0303DBB2002B6D
:1012F00005D04FF001004FF4802101F029FE019B41
:10130000022B14BF00230123DAB2019B032B14BF6D
:1013100000230123DBB242EA0303DBB2002B05D03A
:101320004FF003004FF0806101F012FE4FF0000318
:10133000039303E0039B03F101030393039A4FF626
:10134000FF73C0F20F039A42F4D905B000BD00BF8D
:1013500000B583B04FF001038DF802304FF0000369
:101360008DF804304FF000038DF803304FF00A037E
:101370008DF801304FF002038DF800306B461846AF
:1013800002F0C8FA4CF20003C4F20F034FF000025F
:10139000C3F840214CF20003C4F20F034FF00002E7
:1013A000C3F848214CF20003C4F20F034FF00002CF
:1013B000C3F84C214CF20003C4F20F034FF00F02AC
:1013C000C3F848214CF20003C4F20F034FF00002AF
:1013D000C3F84C214CF20003C4F20F034FF00F028C
:1013E000C3F840214FF012004FF00401FFF7A4FCB6
:1013F0004FF01200FFF788FC03B000BD00B58BB0C2
:101400004FF001038DF816304FF000038DF81830BF
:101410004FF000038DF817304FF001038DF81430B2
:101420004FF000038DF8153005AB184602F072FA44
:101430004FF001038DF8153005AB184602F06AFA3B
:101440004FF004038DF8153005AB184602F062FA30
:101450004FF008038DF8153005AB184602F05AFA24
:101460004FF009038DF8153005AB184602F052FA1B
:101470004FF00A038DF8153005AB184602F04AFA12
:101480004FF00E038DF8153005AB184602F042FA06
:101490004FF00F038DF8153005AB184602F03AFAFD
:1014A0004FF010038DF8153005AB184602F032FAF4
:1014B0004FF011038DF8153005AB184602F02AFAEB
:1014C00043F2A413C1F200031B684CF20000C4F203
:1014D00000004BF2F001C0F20001984740F208030F
:1014E000C1F200031B781A4640F20803C1F2000360
:1014F0005B789C4640F20803C1F200039B789E464D
:1015000040F20803C1F20003DB78184640F20803FA
:10151000C1F200031B79194640F20803C1F200032F
:101520005B79CDF800E001900291039343F24C10F7
:10153000C1F200004BF20411C0F20001634604F056
:1015400005FF43F29C13C1F200031B684CF200003C
:10155000C4F2000043F24C11C1F2000198474FF071
:101560000003079340F20803C1F20003089318E058
:1015700043F2A413C1F200031B684CF20000C4F252
:1015800000004BF22C11C0F2000198474FF4801379
:10159000099303E0099B03F1FF330993099B002B97
:1015A000F8D107AB184601F021F80346002BDFD035
:1015B0004FF0FF004FF0010101F030FB4FF01C0035
:1015C0004FF00001FFF7B8FB4FF01C00FFF79CFB4A
:1015D00043F2A413C1F200031B684CF20000C4F2F2
:1015E00000004BF26411C0F2000198470BB000BD3F
:1015F00000B589B04FF0000306934BF2BC12C0F265
:10160000000201AB92E80300186003F104031980A3
:101610004FF00400FFF750FBFEF7F4FF00F068FD09
:10162000FFF716F9FFF7BEF843F2C803C1F2000353
:1016300005930598FEF750FF01AB18464FF00101E6
:1016400001F0ECF943F2A413C1F200031B684CF261
:101650000000C4F200004BF28011C0F20001984774
:101660004FF440504FF0010101F02AFA4FF000030F
:10167000069307E04FF00100FFF714F8069B03F113
:1016800001030693069B042BF4D972B64CF20003B7
:10169000C4F20F034FF00002C3F8C02030BF03F0C4
:1016A000CFFE00F025FDFEF7ADFF43F2A413C1F21B
:1016B00000031B684CF20000C4F200004BF29811CA
:1016C000C0F200019847FFF7C3F862B603E04FF09D
:1016D0000300FEF7E7FF40F26153C1F200031B78FD
:1016E000DBB2002BF3D040F26153C1F200034FF0A4
:1016F00000021A7043F2C803C1F20003059343F2DB
:10170000A413C1F200031B684CF20000C4F20000F5
:101710004BF2B011C0F2000198474FF00200FEF703
:10172000C1FF059B04934FF07603039303AB184668
:1017300001F002FA01F01CFB4FF00003079303E0F5
:10174000079B03F101030793079A4FF6FF73C0F25B
:101750001F039A42F4D900BFBDE700BF08B5FFF7E9
:1017600071F90346184608BD82B001900091FEE76A
:1017700082B001904FF0FF33184602B0704700BFAF
:1017800084B003900291019243F2B413C1F20003BA
:101790004FF00C021A604FF0FF33184604B0704748
:1017A0004FF000031846704743F2B413C1F2000330
:1017B0004FF00B021A604FF0FF331846704700BF1E
:1017C00082B001900091009B4FF400525A604FF09C
:1017D0000003184602B070474FF0010318467047E7
:1017E00082B00190009143F2B413C1F200034FF0B4
:1017F00016021A604FF0FF33184602B0704700BF60
:1018000082B001904FF00103184602B0704700BF4C
:1018100082B001904FF00103184602B0704700BF3C
:1018200082B00190009143F2B413C1F200034FF073
:101830001F021A604FF0FF33184602B0704700BF16
:1018400084B00390029101924FF00003184604B057
:10185000704700BF84B00390029101924FF0FF33B4
:10186000184604B0704700BF84B003900291019203
:101870004FF00003184604B0704700BF84B00190D9
:1018800040F29853C1F200031B68002B14D140F2C0
:101890009853C1F2000348F20002C1F200021A603C
:1018A00040F29853C1F200031B6803F5804240F2F6
:1018B0009853C1F200031A6040F29853C1F200033A
:1018C0001B68039340F29853C1F200031A68019B0E
:1018D0001A4440F29853C1F200031A60039B184661
:1018E00004B0704782B001900091009B4FF4005209
:1018F0005A604FF00003184602B0704782B0019062
:101900004FF0FF33184602B0704700BF82B001901D
:1019100043F2B413C1F200034FF002021A604FF019
:10192000FF33184602B0704782B0019043F2B413FF
:10193000C1F200034FF00A021A604FF0FF3318465D
:1019400002B0704784B00390029101924FF00003FF
:10195000184604B0704700BF82B001900091FEE7C6
:10196000FEE7FEE7FEE7FEE7FEE7FEE7FEE7FEE74F
:10197000FEE7FEE700B583B001900B468DF803301B
:101980000DF10303019819464FF001024FF00103D6
:1019900002F006FC03B000BD00B585B001904FF029
:1019A00000038DF80F300DF10F03019819464FF029
:1019B00001024FF0010302F077FC9DF80F3018464A
:1019C00005B000BD00B585B001900091009B039368
:1019D00009E0039B1B78039A02F10102039201982C
:1019E0001946FFF7C7FF039B1B78002BF1D105B009
:1019F00000BD00BF00B583B001900091019800992F
:101A0000FFF7E0FF01984BF2C411C0F20001FFF7AD
:101A1000D9FF03B000BD00BF00B585B001900B46F3
:101A20008DF803309DF803204CF6CD43CCF6CC4323
:101A3000A3FB02134FEAD3010B464FEA83030B4487
:101A40004FEA4303C3EB02038DF80D309DF80320EA
:101A50004CF6CD43CCF6CC43A3FB02134FEAD303A1
:101A6000DAB24CF6CD43CCF6CC43A3FB02134FEADB
:101A7000D3010B464FEA83030B444FEA4303C3EB06
:101A800002038DF80E309DF8032048F21F53C5F273
:101A9000EB13A3FB02134FEA5313DAB24CF6CD4318
:101AA000CCF6CC43A3FB02134FEAD3010B464FEA1B
:101AB00083030B444FEA4303C3EB02038DF80F305B
:101AC0009DF80F3003F13003DBB201981946FFF7A0
:101AD00051FF9DF80E3003F13003DBB20198194637
:101AE000FFF748FF9DF80D3003F13003DBB201989A
:101AF0001946FFF73FFF05B000BD00BF00B585B038
:101B000001900B46ADF80230BDF802204CF6CD43F3
:101B1000CCF6CC43A3FB02134FEAD3010B464FEAAA
:101B200083030B444FEA4303C3EB02039BB28DF8DC
:101B30000B30BDF802204CF6CD43CCF6CC43A3FBD2
:101B400002134FEAD3039AB24CF6CD43CCF6CC4302
:101B5000A3FB02134FEAD3010B464FEA83030B4466
:101B60004FEA4303C3EB02039BB28DF80C30BDF880
:101B7000022048F21F53C5F2EB13A3FB02134FEAF6
:101B800053139AB24CF6CD43CCF6CC43A3FB0213CD
:101B90004FEAD3010B464FEA83030B444FEA43035A
:101BA000C3EB02039BB28DF80D30BDF8022044F662
:101BB000D353C1F26203A3FB02134FEA93139AB209
:101BC0004CF6CD43CCF6CC43A3FB02134FEAD30132
:101BD0000B464FEA83030B444FEA4303C3EB020374
:101BE0009BB28DF80E30BDF8022041F25973CDF250
:101BF000B713A3FB02134FEA53339AB24CF6CD430B
:101C0000CCF6CC43A3FB02134FEAD3010B464FEAB9
:101C100083030B444FEA4303C3EB02039BB28DF8EB
:101C20000F309DF80F3003F13003DBB201981946F5
:101C3000FFF7A0FE9DF80E3003F13003DBB20198F0
:101C40001946FFF797FE9DF80D3003F13003DBB224
:101C500001981946FFF78EFE9DF80C3003F1300312
:101C6000DBB201981946FFF785FE9DF80B3003F1B2
:101C70003003DBB201981946FFF77CFE05B000BDCA
:101C800000B587B00190009100994CF6CD43CCF699
:101C9000CC43A3FB01234FEAD30213464FEA83034D
:101CA00013444FEA4303C3EB010213468DF80E3091
:101CB000009A4CF6CD43CCF6CC43A3FB02134FEA7B
:101CC000D3014CF6CD43CCF6CC43A3FB01234FEA22
:101CD000D30213464FEA830313444FEA4303C3EB93
:101CE000010213468DF80F30009A48F21F53C5F2D7
:101CF000EB13A3FB02134FEA53114CF6CD43CCF682
:101D0000CC43A3FB01234FEAD30213464FEA8303DC
:101D100013444FEA4303C3EB010213468DF810301E
:101D2000009A44F6D353C1F26203A3FB02134FEAB5
:101D300093114CF6CD43CCF6CC43A3FB01234FEAE1
:101D4000D30213464FEA830313444FEA4303C3EB22
:101D5000010213468DF81130009A41F25973CDF209
:101D6000B713A3FB02134FEA53314CF6CD43CCF625
:101D7000CC43A3FB01234FEAD30213464FEA83036C
:101D800013444FEA4303C3EB010213468DF81230AC
:101D9000009B4FEA531245F6C523C0F67C23A3FBF4
:101DA00002134FEAD3114CF6CD43CCF6CC43A3FB40
:101DB00001234FEAD30213464FEA830313444FEA49
:101DC0004303C3EB010213468DF81330009A4DF61E
:101DD0008363C4F21B33A3FB02134FEA93414CF617
:101DE000CD43CCF6CC43A3FB01234FEAD3021346E9
:101DF0004FEA830313444FEA4303C3EB0102134644
:101E00008DF81430009A4CF66B23C6F65F33A3FBB3
:101E100002134FEA93514CF6CD43CCF6CC43A3FBCF
:101E200001234FEAD30213464FEA830313444FEAD8
:101E30004303C3EB010213468DF81530009A43F6B5
:101E40008933C5F2E653A3FB02134FEA53614CF604
:101E5000CD43CCF6CC43A3FB01234FEAD302134678
:101E60004FEA830313444FEA4303C3EB01021346D3
:101E70008DF81630009B4FEA532244F68333C0F2AC
:101E80000403A3FB02134FEAD3114CF6CD43CCF667
:101E9000CC43A3FB01234FEAD30213464FEA83034B
:101EA00013444FEA4303C3EB010213468DF8173086
:101EB0009DF8173003F13003DBB201981946FFF7A4
:101EC00059FD9DF8163003F13003DBB20198194635
:101ED000FFF750FD9DF8153003F13003DBB2019898
:101EE0001946FFF747FD9DF8143003F13003DBB2CC
:101EF00001981946FFF73EFD9DF8133003F13003BA
:101F0000DBB201981946FFF735FD9DF8123003F159
:101F10003003DBB201981946FFF72CFD9DF8113014
:101F200003F13003DBB201981946FFF723FD9DF85A
:101F3000103003F13003DBB201981946FFF71AFDA8
:101F40009DF80F3003F13003DBB201981946FFF71B
:101F500011FD9DF80E3003F13003DBB201981946F4
:101F6000FFF708FD07B000BD00B585B001900B4636
:101F70008DF8033001984BF2C811C0F20001FFF751
:101F800021FD4FF001038DF80F309DF803209DF8DF
:101F90000F304FEA830342FA03F3DBB203F00F037F
:101FA0008DF80E309DF80E30092B05D99DF80E30B6
:101FB00003F13703DBB204E09DF80E3003F1300388
:101FC000DBB201981946FFF7D5FC9DF80F30002BC6
:101FD0000CBF00230123DBB29DF80F2002F1FF327A
:101FE0008DF80F20002BD0D105B000BD00B585B015
:101FF00001900B46ADF8023001984BF2C811C0F2C7
:102000000001FFF7DFFC4FF003038DF80F30BDF840
:1020100002209DF80F304FEA830342FA03F3DBB24C
:1020200003F00F038DF80E309DF80E30092B05D903
:102030009DF80E3003F13703DBB204E09DF80E305B
:1020400003F13003DBB201981946FFF793FC9DF8CA
:102050000F30002B0CBF00230123DBB29DF80F20B3
:1020600002F1FF328DF80F20002BD0D105B000BD5A
:1020700000B585B00190009101984BF2C811C0F2F3
:102080000001FFF79FFC4FF007038DF80F309DF81C
:102090000F304FEA8303009A22FA03F3DBB203F016
:1020A0000F038DF80E309DF80E30092B05D99DF8E1
:1020B0000E3003F13703DBB204E09DF80E3003F17C
:1020C0003003DBB201981946FFF754FC9DF80F303E
:1020D000002B0CBF00230123DBB29DF80F2002F17F
:1020E000FF328DF80F20002BD1D105B000BD00BF0D
:1020F00000B585B04FF001038DF802304FF00003BA
:102100008DF804304FF000038DF803304FF00203D8
:102110008DF801304FF000038DF800306B46184603
:1021200001F0F8FB4FF003038DF801306B461846C1
:1021300001F0F0FB02AB184601F0AAFF4FF4E133C7
:10214000029302AB4CF20000C4F20000194601F009
:1021500091FD4CF20000C4F200004FF0010102F0CA
:10216000A5FC43F29C13C1F2000341F6C512C0F274
:1021700000021A6043F2A413C1F2000341F6F51203
:10218000C0F200021A6043F2A813C1F2000341F644
:102190007512C0F200021A6043F2AC13C1F20003E0
:1021A00041F66972C0F200021A6043F2B013C1F244
:1021B000000341F6ED72C0F200021A6043F294137C
:1021C000C1F2000342F27102C0F200021A6043F24F
:1021D0008C13C1F2000341F61922C0F200021A600A
:1021E00043F29813C1F2000341F6FD22C0F200024F
:1021F0001A6043F29013C1F2000341F68142C0F22B
:1022000000021A6043F2A013C1F2000341F69912D2
:10221000C0F200021A6005B000BD00BF82B04FF0EE
:102220000003019339E00199019A13464FEA4303F1
:1022300013444FEA43231A4640F20463C1F20003F9
:1022400013441A4640F29C53C1F2000343F8312074
:10225000019B40F29C52C1F200024FEAC3031344B7
:1022600040F2FF52C8F200025A60019A40F2C05395
:10227000C1F200034FF0000143F83210019B40F21D
:10228000C052C1F200024FEAC30313444FF00002F0
:102290005A60019B03F101030193019B032BC2D9F7
:1022A0004FF0A04240F29C53C1F20003C2F8083143
:1022B0004FF0A04240F2C053C1F20003C2F80C310B
:1022C0004FF0A0434FF00302C3F810214FF0A0439A
:1022D0004FF00002C3F8182102B0704782B04FF0EF
:1022E000000301932CE00199019A13464FEA43033E
:1022F00013444FEA43231A4641F60463C1F2000334
:1023000013441A4640F2E053C1F2000343F831206F
:10231000019B40F2E052C1F200024FEAC3031344B2
:102320004FF000025A60019A40F2F853C1F20003E4
:102330004FF0000143F82210019B03F101030193C8
:10234000019B022BCFD94FF0A04240F2E053C1F2E3
:102350000003C2F81C314FF0A04240F2F853C1F222
:102360000003C2F820314FF0A0434FF00202C3F83F
:1023700024214FF0A0434FF00002C3F8282102B0FF
:10238000704700BF84B001900B46ADF802304FF0AB
:10239000A043019A42F480729A624FF0A043BDF8C4
:1023A0000220DA624FF0000303934FF0000303931F
:1023B0000DE04FF0A0435B6B03F00103002B02D153
:1023C0004FF000030CE0039B03F101030393039A16
:1023D0004FF6FF73C0F204039A42EAD94FF0FF337D
:1023E000184604B0704700BF84B001904FF0A0437E
:1023F000019A42F480729A624FF0A0434FF00102BA
:102400005A624FF0000303934FF00003039313E06D
:102410004FF0A0435B6B03F00103002B08D14FF09A
:10242000A0434FF000025A624FF0A0431B6B0CE038
:10243000039B03F101030393039A4FF6FF73C0F26A
:1024400004039A42E4D94FF0FF33184604B07047B2
:1024500082B001904FF0A043019A02F10502127878
:102460004FEA0221019A02F10402127841EA0202C3
:102470001A644FF0A043019A02F1030212784FEA66
:102480000221019A02F10202127841EA02025A6420
:102490004FF0A043019A02F1010212784FEA0221A3
:1024A000019A127841EA02029A6402B0704700BFB2
:1024B0008AB0019000914FF0FF3305934FF0000375
:1024C000029389E0019B1B788DF81330019B03F187
:1024D000010301934FF00003039376E0059B4FEA5D
:1024E00023729DF813304FEAD303DBB282EA030371
:1024F00003F00103DBB2002B05D041F6B753C0F265
:10250000C143099302E04FF000030993059B4FEA92
:1025100063729DF813304FEA9303DBB282EA030340
:1025200003F00103DBB2002B05D043F66E33C0F697
:102530008213089302E04FF000030893059B4FEAD3
:10254000A3729DF813304FEA5303DBB282EA030310
:1025500003F00103DBB2002B05D047F2DC63C1F2CC
:102560000433079302E04FF000030793059B4FEA03
:10257000E3729DF8133082EA030303F00103DBB238
:10258000002B05D04EF6B853C2F20863069302E062
:102590004FF000030693059B4FEA0312099B82EA62
:1025A0000302089B82EA0302079B82EA0302069B5E
:1025B00082EA030305939DF813304FEA13138DF855
:1025C0001330039B03F101030393039B012B85DD70
:1025D000029B03F101030293029A009B9A42FFF6C9
:1025E00071AF059B18460AB0704700BF00B587B0B1
:1025F00001904FF080404FF0010103F0F3F84FF0ED
:10260000A0434FF44F421A604FF0A0434FF07802BE
:10261000C3F800214FF06403049303E0049B03F12B
:10262000FF330493049B002BF8D14FF0A0434FF0ED
:1026300002021A604FF0A0434FF030025A604FF090
:10264000A0434FF4C0625A6140F21C03C1F2000380
:102650001A684CF66B23C6F65F33A3FB02134FEAEE
:10266000135305934FF0000304930DE0049A4BF2CB
:10267000CC13C0F200039B5C1A46059B9A4207DA12
:10268000049B03F101030493049B062BEED900E0A5
:1026900000BF049B03F1010304934FF0A043049A8D
:1026A00002F00F024FEA820242F400421A624FF037
:1026B000A0434FF0A042126A22F400421A624FF087
:1026C000A04343F20F721A614FF0A0434FF0120281
:1026D000DA604FF0A0434FF41072C3F800214FF0BE
:1026E000A0434FF400629A614FF06403049303E047
:1026F000049B03F1FF330493049B002BF8D14FF0AC
:10270000A0434FF000029A614FF000004FF40041E7
:10271000FFF738FE4FF48013049314E04FF00000ED
:10272000FFF762FE03460393039B03F40843002B69
:102730000DD0049B002B02D14FF0000342E0049B1C
:1027400003F1FF330493049B002BE7D100E000BFAB
:10275000019B1B68184600F081F80346002B02DA43
:102760004FF000032EE0019B5B681846FFF770FEF8
:10277000FFF754FDFFF7B2FD4FF0A0434FF02602E4
:10278000C3F800224FF0A0434FF08802C3F8E42FB3
:102790004FF0A0434FF6FF72C3F8E82F4FF0A0436D
:1027A0004FF0A042D2F8002142F00302C3F800210A
:1027B0004FF0A0434FF0A042126842F001021A60AD
:1027C0004FF00103184607B000BD00BF08B54FF039
:1027D000A0434FF00002C3F8E42F4FF0A04343F2B0
:1027E000FF02C3F8E82F4FF080404FF0000102F0E5
:1027F000F9FF08BD00B585B001904FF00100FFF76B
:10280000F3FD03460293019B012B0DD0012B02D354
:10281000022B12D01AE0029B03F00403002B0CBF22
:1028200000230123039314E0029B03F4C043002B15
:102830000CBF0023012303930BE0029B03F4A0438E
:10284000002B0CBF00230123039302E04FF0FF3362
:102850000393039B184605B000BD00BF00B587B0C9
:1028600001904FF00200FFF7BFFD034602934FF0C7
:102870000300FFF7B9FD03460393029B4FEA0342AF
:10288000039B42EA030241F21353C0F222039A422D
:1028900060D1019B042B54D801A252F823F000BF51
:1028A000B52800000B290000192900002729000085
:1028B000352900004FF000004FF44051FFF762FD52
:1028C0004FF000004FF48051FFF75CFD4FF4801390
:1028D000049316E04FF00100FFF786FD03460593D1
:1028E000059B03F02003002B01D000BF2CE0049BCC
:1028F000002B02D14FF0FF3334E0049B03F1FF3390
:102900000493049B002BE5D11EE04FF000004FF430
:102910008071FFF737FD17E04FF000004FF0000126
:10292000FFF730FD10E04FF000004FF40451FFF7C7
:1029300029FD09E04FF000004FF40051FFF722FDA0
:1029400002E04FF0FF330DE000F010F80346002BDB
:1029500003DB05E04FF0FF3304E04FF0FF3301E00D
:102960004FF00003184607B000BD00BF00B583B0AC
:102970004FF48013019314E04FF00100FFF734FD92
:1029800003460093009B03F00403002B0DD1019B31
:10299000002B02D14FF0FF333CE0019B03F1FF33EA
:1029A0000193019B002BE7D100E000BF009B03F4E3
:1029B000A043002B17D04FF0A0434FF0A042526825
:1029C00042F001025A604FF0A0434FF0A042D2F80B
:1029D000002142F48062C3F800214FF0A0434FF081
:1029E00015029A6004E04FF0A0434FF012029A6083
:1029F000009B03F4C043002B05D14FF0A0434FF0E0
:102A000000029A6104E04FF0A0434FF480729A6193
:102A10004FF00003184603B000BD00BF00B587B0FB
:102A200001900B468DF8033001984FF00601FFF737
:102A30003FFD03460593059B4FEAE35303F03F0335
:102A40000593059B1F2B04DD40F21423C5F2000300
:102A500003E040F21023C5F200030393059B1F2BF4
:102A600003DD059BA3F1200300E0059B04939DF883
:102A70000330012B0BD1039B1A68049B4FF001011B
:102A800001FA03F342EA0302039B1A600CE0039B82
:102A90001A68049B4FF0010101FA03F36FEA030384
:102AA00002EA0302039B1A604FF0A0434FF0A042DA
:102AB000D2F8002122F08002C3F8002107B000BD47
:102AC00082B001900B468DF803309DF80330012B46
:102AD0000BD14FF0A0434FF0A042D2F80012019A60
:102AE00041EA0202C3F800220CE04FF0A0434FF08D
:102AF000A042D2F80012019A6FEA020201EA020231
:102B0000C3F8002202B0704782B001904FF0A0439A
:102B1000D3F80422019B02EA0303002B07D04FF0F5
:102B2000A043019AC3F808224FF0010301E04FF0DF
:102B30000003184602B0704786B001904FF0A043E2
:102B4000D3F828310293019B5B680493029A40F208
:102B5000E053C1F2000353F832300593019B1B6828
:102B600003F103034FEA930303930FE0049B1A68F6
:102B7000059B1A60059B03F104030593049B03F175
:102B800004030493039B03F1FF330393039B002B84
:102B9000ECD1029B019A126802F1FF3242F04041EF
:102BA00040F2E052C1F200024FEAC30313445960FD
:102BB00006B0704786B001904FF0A043D3F81831AB
:102BC0000293019B5B680493029A40F29C53C1F20A
:102BD000000353F832300593019B5B68002B1AD039
:102BE000019B1B6803F103034FEA930303930FE078
:102BF000059B1A68049B1A60049B03F10403049369
:102C0000059B03F104030593039B03F1FF33039337
:102C1000039B002BECD106B0704700BF82B001903F
:102C20000B468DF803309DF80330012B0BD14FF08C
:102C3000A0434FF0A042D2F8E41F019A41EA0202F9
:102C4000C3F8E42F0CE04FF0A0434FF0A042D2F8BD
:102C5000E41F019A6FEA020201EA0202C3F8E42FBC
:102C600002B0704782B001904FF0A043D3F8E02F3C
:102C7000019B02EA0303002B07D04FF0A043019A07
:102C8000C3F8E82F4FF0010301E04FF000031846AE
:102C900002B070474FF0A043D3F818214FF0A04383
:102CA000D3F814319A4202D04FF0010301E04FF003
:102CB00000031846704700BF82B04FF0A043D3F81E
:102CC0002C3103F1FF3301934FF0A043D3F82821B7
:102CD000019B9A4202D14FF0000301E04FF0010343
:102CE000184602B0704700BF84B001904FF0A04377
:102CF000D3F818310393039A40F2C053C1F2000392
:102D000053F83220019B02EA0303002B0CBF00237F
:102D10000123184604B0704782B04FF0A043D3F8A7
:102D200018310193019A40F2C053C1F2000353F8E5
:102D300032304FEA43534FEA5353184602B07047BC
:102D400082B04FF0A043D3F818310193019B03F1F7
:102D500001030193019B042B02D14FF00003019367
:102D60004FF0A043019AC3F8182102B0704700BF8A
:102D700082B04FF0A043D3F828310193019B03F1B7
:102D800001030193019B032B02D14FF00003019338
:102D90004FF0A043019AC3F8282102B0704700BF4A
:102DA00084B003468DF807304FF0000303939DF87D
:102DB0000730042B29D801A252F823F0D12D0000AE
:102DC000DD2D0000E92D0000F52D0000012E000092
:102DD0004CF20003C2F20903039316E04CF2200305
:102DE000C2F20903039310E04CF24003C2F209035C
:102DF00003930AE04CF26003C2F20903039304E078
:102E00004CF28003C2F209030393039B184604B0FB
:102E1000704700BF84B003468DF807304FF00003C1
:102E200003939DF80730042B29D801A252F823F010
:102E3000452E0000512E00005D2E0000692E00007E
:102E4000752E00004CF20003C2F20903039316E052
:102E50004CF22003C2F20903039310E04CF240034A
:102E6000C2F2090303930AE04CF26003C2F20903C1
:102E7000039304E04CF28003C2F209030393039B23
:102E8000184604B0704700BF84B003468DF8073081
:102E90004FF0000303939DF80730042B29D801A2BB
:102EA00052F823F0B92E0000C52E0000D12E0000EC
:102EB000DD2E0000E92E00004CF20003C2F20903EF
:102EC000039316E04CF22003C2F20903039310E0CF
:102ED0004CF24003C2F2090303930AE04CF2600390
:102EE000C2F20903039304E04CF28003C2F2090327
:102EF0000393039B184604B0704700BF00B587B02A
:102F00000291134602468DF80F208DF807309DF888
:102F10000F301846FFF744FF03460593059B002B2F
:102F200014D09DF80730002B07D0059B1A68029B30
:102F300042EA0302059B1A6008E0059B1A68029B9F
:102F40006FEA030302EA0302059B1A6007B000BDA3
:102F500000B585B0034600918DF807309DF8073025
:102F60001846FFF71DFF03460393039B002B02D077
:102F7000039B009A9A6105B000BD00BF00B585B003
:102F8000034600918DF807309DF807301846FFF78B
:102F900007FF03460393039B002B02D0039B009A79
:102FA000DA6105B000BD00BF00B585B003468DF8FD
:102FB00007309DF807301846FFF7F2FE03460393EB
:102FC000039B002B02D0039B5B6901E04FF00003E1
:102FD000184605B000BD00BF84B0029113460246FA
:102FE0008DF80F208DF807309DF80F30002B0AD197
:102FF0009DF80730002B06D148F28003C4F202038B
:10300000029A1A612EE09DF80F30022B0AD19DF82A
:103010000730002B06D148F28003C4F20203029A63
:103020001A631FE09DF80F30002B0AD19DF807307E
:10303000012B06D148F28003C4F20203029A5A61BE
:1030400010E09DF80F30022B0BD19DF80730012BBB
:1030500007D148F28003C4F20203029A5A6300BF08
:1030600000E0FEE704B0704784B0029113460246C8
:103070008DF80F208DF807309DF80F30002B0FD101
:103080009DF80730002B0BD148F28003C4F20203F5
:103090005A68029B22FA03F3DBB203F001033CE01F
:1030A0009DF80F30022B0FD19DF80730002B0BD16C
:1030B00048F28003C4F202035A6A029B22FA03F325
:1030C000DBB203F0010328E09DF80F30002B0FD195
:1030D0009DF80730012B0BD148F28003C4F20203A4
:1030E0009A68029B22FA03F3DBB203F0010314E0B7
:1030F0009DF80F30022B0FD19DF80730012B0BD11B
:1031000048F28003C4F202039A6A029B22FA03F394
:10311000DBB203F0010300E0FEE7184604B070479D
:1031200082B0034600918DF807309DF80730002BE0
:1031300006D148F28003C4F20203009ADA600BE081
:103140009DF80730022B06D148F28003C4F2020337
:10315000009ADA6200E0FEE702B0704700B585B081
:103160000291134602468DF80F208DF807309DF826
:103170000F209DF80730104602991A46FFF7BEFE51
:1031800005B000BD00B583B0034600918DF807304F
:103190009DF8073018460099FFF7DAFE03B000BD2E
:1031A00000B583B0034600918DF807309DF80730D5
:1031B00018460099FFF7E2FE03B000BD00B583B0EA
:1031C00003468DF807309DF807301846FFF7ECFEF0
:1031D0000346184603B000BD00B585B00291134602
:1031E00002468DF80F208DF807309DF80F209DF8CE
:1031F0000730104602991A46FFF7EEFE05B000BDF3
:1032000000B585B00291134602468DF80F208DF867
:1032100007309DF80F209DF80730104602991A4696
:10322000FFF722FF0346184605B000BD00B583B086
:10323000034600918DF807309DF807301846009935
:10324000FFF76EFF03B000BD00B587B002911346D3
:1032500002468DF80F208DF807309DF80F30184684
:10326000FFF79EFD03460593059B002B14D09DF8A8
:103270000730002B07D0059B1A69029B42EA030224
:10328000059B1A6108E0059B1A69029B6FEA03031C
:1032900002EA0302059B1A6107B000BD00B585B0C4
:1032A0008DF807008DF80610ADF804208DF8033076
:1032B0009DF807301846FFF7ADFD03460393039BC7
:1032C000002B40D09DF80330002B19D09DF806301C
:1032D000002B0AD0039B5B889AB2BDF8043042EA07
:1032E00003039AB2039B5A802DE0039B1B889AB27A
:1032F000BDF8043042EA03039AB2039B1A8022E02D
:103300009DF80630002B0FD0039B5B889BB21A46BA
:10331000BDF804306FEA03039BB202EA03039BB2D9
:103320009AB2039B5A800EE0039B1B889BB21A46FD
:10333000BDF804306FEA03039BB202EA03039BB2B9
:103340009AB2039B1A8005B000BD00BF00B585B0DE
:103350008DF807008DF80610ADF804208DF80330C5
:103360009DF807301846FFF755FD03460393039B6E
:10337000002B40D09DF80330002B19D09DF806306B
:10338000002B0AD0039B5B8A9AB2BDF8043042EA54
:1033900003039AB2039B5A822DE0039B1B8A9AB2C5
:1033A000BDF8043042EA03039AB2039B1A8222E07A
:1033B0009DF80630002B0FD0039B5B8A9BB21A4608
:1033C000BDF804306FEA03039BB202EA03039BB229
:1033D0009AB2039B5A820EE0039B1B8A9BB21A4649
:1033E000BDF804306FEA03039BB202EA03039BB209
:1033F0009AB2039B1A8205B000BD00BF00B585B02C
:10340000134602468DF807200A468DF80620ADF8CF
:1034100004309DF807301846FFF7FCFC0346039381
:10342000039B002B0CD09DF80630002B04D0039B8F
:10343000BDF804205A8303E0039BBDF804201A83DF
:1034400005B000BD00B585B0134602468DF80720D3
:103450000A468DF80620ADF804309DF8073018466E
:10346000FFF7D8FC03460393039B002B0CD09DF879
:103470000630002B04D0039BBDF80420DA8303E060
:10348000039BBDF804209A8305B000BD00B585B04C
:1034900002460B468DF807208DF806309DF8073060
:1034A0001846FFF7B7FC03460393039B002B0BD092
:1034B0009DF80630002B03D0039BDB8A9BB205E00E
:1034C000039B9B8A9BB201E04FF00003184605B0B6
:1034D00000BD00BF00B585B08DF807008DF806105F
:1034E0008DF805208DF804309DF807301846FFF759
:1034F000CBFC03460393039B002B2FD09DF8043095
:10350000002B12D09DF80630032B26D89DF80630EC
:103510009DF8062003998A5CD1B29DF8052041EA06
:103520000202D1B2039AD15418E09DF80630032B61
:1035300014D89DF806309DF8062003998A5CD2B213
:1035400011469DF805206FEA0202D2B201EA02029A
:10355000D2B2D1B2039AD15400E000BF05B000BD91
:1035600000B585B08DF807008DF806108DF80520A0
:103570008DF804309DF807301846FFF785FC0346A8
:103580000393039B002B33D09DF80430002B14D001
:103590009DF80630032B2AD89DF806109DF80620CA
:1035A000039B13441B7CDAB29DF8053042EA030307
:1035B000DAB2039B0B441A741AE09DF80630032B11
:1035C00016D89DF806109DF80620039B13441B7C1B
:1035D000DBB21A469DF805306FEA0303DBB202EA5C
:1035E0000303DBB2DAB2039B0B441A7400E000BFA2
:1035F00005B000BD00B585B0134602468DF8072022
:103600000A468DF806208DF805309DF807301846DB
:10361000FFF73AFC03460393039B002B0AD09DF867
:103620000630032B06D89DF80620039B13449DF813
:1036300005201A7605B000BD00B585B013460246D8
:103640008DF807200A468DF806208DF805309DF884
:1036500007301846FFF718FC03460393039B002B23
:103660000AD09DF80630032B06D89DF80620039B50
:1036700013449DF805201A7705B000BD00B585B04C
:1036800002460B468DF807208DF806309DF807306E
:103690001846FFF7F9FB03460393039B002B0AD060
:1036A0009DF80630032B06D89DF80620039B134493
:1036B0001B7DDBB201E04FF00003184605B000BDF2
:1036C00086B0134602468DF807200A468DF806207C
:1036D0008DF805309DF8063003939DF807304FEACA
:1036E000430304934CF20003C4F202030593039BCB
:1036F0000F2B07D9039BA3F110030393049B03F142
:1037000001030493049B4FEA8302059B1344049A2C
:103710004FEA8201059A0A441168039A4FEA42026D
:103720004FF0030000FA02F26FEA020201EA02021D
:103730001A60049B4FEA8302059B1344049A4FEAE4
:103740008201059A0A4411689DF80500039A4FEA20
:10375000420200FA02F241EA02021A6006B0704721
:1037600086B0134602468DF807200A468DF80620DB
:103770008DF805309DF8063003939DF807304FEA29
:10378000430304934CF24003C4F202030593039BEA
:103790000F2B07D9039BA3F110030393049B03F1A1
:1037A00001030493049B4FEA8302059B1344049A8C
:1037B0004FEA8201059A0A441168039A4FEA4202CD
:1037C0004FF0030000FA02F26FEA020201EA02027D
:1037D0001A60049B4FEA8302059B1344049A4FEA44
:1037E0008201059A0A4411689DF80500039A4FEA80
:1037F000420200FA02F241EA02021A6006B0704781
:1038000084B0134602468DF807200A468DF806203C
:103810008DF805304CF26803C4F2020303939DF85F
:103820000530012B16D19DF807304FEA8302039B28
:1038300013449DF807204FEA8201039A0A44116855
:103840009DF806204FF0010000FA02F241EA020260
:103850001A6017E09DF807304FEA8302039B134478
:103860009DF807204FEA8201039A0A4411689DF8E7
:1038700006204FF0010000FA02F26FEA020201EAAC
:1038800002021A6004B0704782B003468DF8073018
:103890009DF80730012B0CD14CF20003C4F2020357
:1038A0004CF20002C4F20202926A42F008029A62EA
:1038B0000FE09DF80730002B0BD14CF20003C4F24F
:1038C00002034CF20002C4F20202926A22F00802E1
:1038D0009A6202B0704700BF84B002460B468DF872
:1038E00007208DF806309DF80730012B02D14FF0EC
:1038F000050303939DF80630002B02D14FF00A0315
:1039000003934CF20003C4F20203039ADA6704B093
:10391000704700BF00B583B00190019B1978019BEF
:103920005A78019B9B78084611461A46FFF7C8FE55
:10393000019B1978019B5A78019BDB780846114658
:103940001A46FFF70DFF019B1978019B5A78019BDE
:103950001B79084611461A46FFF752FF03B000BD17
:103960002DE9F04F95B0039002914FF000038DF8D0
:103970001730039A4CF20003C4F200039A4206D1B6
:103980004FF0060001F0FAFE0346069328E0039A82
:1039900040F20003C4F201039A4206D14FF008003E
:1039A00001F0ECFE034606931AE0039A48F2000386
:1039B000C4F209039A4206D14FF0300001F0DEFE56
:1039C000034606930CE0039A4CF20003C4F2090389
:1039D0009A4205D14FF0320001F0D0FE0346069323
:1039E0004FF0FF3312934FF0000309934FF00003A1
:1039F0000A934FF000024FF00003CDE90C234FF083
:103A00000103089374E04FF00003079363E0069B03
:103A10001A464FF000034FEA12114FEA037541EACC
:103A200005054FEA0274089B1A464FF0000302FB9B
:103A300005F104FB03F00144A4FB022319440B46E7
:103A4000089807990144029800FB01F18A464FF05B
:103A5000000BCDE900AB10461946DDE9002301F06B
:103A60003DFF02460B46CDE90E230E9B11930F9BA3
:103A70009A464FF0000B53460B93119BB3F1004F46
:103A800007D9119BC3F1000311930B9B03F10103B1
:103A90000B930B9B002B17D00B9BB3F5803F15D8D6
:103AA000119A129B9A4212D2119B12930B9B1A46A7
:103AB0004FF00003CDE90C23079B0993089B0A9361
:103AC000129B002B0CD002E000BF00E000BF079B60
:103AD00003F101030793079A089B9A4297D300E0EA
:103AE00000BF129B002B07D0089B03F10103089332
:103AF000089B0F2B87D900E000BFDDE90C2352EAB9
:103B0000030B02D14FF00003AFE0069B4FEA131303
:103B10000A9A02FB03F31C464FF000050A9A099B20
:103B200013441A464FF000030C9903FB01F10D9862
:103B300002FB00F001440C98A0FB022319440B4641
:103B40002046294601F0CAFE02460B46134613934F
:103B5000029A139B9A4205D9029A139BC3EB020364
:103B6000129304E0139A029BC3EB02031293129B7D
:103B70004FF0640202FB03F2029BB2FBF3F31293D9
:103B8000129B022B6FD8039A40F20003C4F2010388
:103B90009A4232D1039A039B1B7BDBB26FEA4363E9
:103BA0006FEA5363DBB21373039B0D9A4FEA026211
:103BB0000C994FEA112842EA08080D9A4FEA122997
:103BC0005FFA88F21A71039B9DF830201A70039AED
:103BD000039B1B7BDBB203F07F031373039B0A9AE7
:103BE0004FEA021202F0FF01099A02F00F0241EAC5
:103BF000020202F0FF029A6231E0039B1B7BDBB200
:103C00006FEA43636FEA5363DAB2039B1A730D9B47
:103C10004FEA03630C9A4FEA122643EA06060D9B0D
:103C20004FEA1327F2B2039B1A719DF83020039BD1
:103C30001A70039B1B7BDBB203F07F03039A1373A1
:103C40000A9BDBB24FEA0313DAB2099BDBB203F043
:103C50000F0342EA0303DAB2039B83F828204FF0F4
:103C600001038DF817309DF81730184615B0BDE8E0
:103C7000F08F00BF00B585B001900091019A4CF221
:103C80000003C4F200039A421CD0019A40F20003E0
:103C9000C4F201039A4215D0019A48F20003C4F21B
:103CA00009039A420ED0019A4CF20003C4F20903B0
:103CB0009A4207D04BF2D410C0F200004FF0CA0174
:103CC000FCF77CFF009B5B79002B13D0009B5B799A
:103CD000012B0FD0009B5B79022B0BD0009B5B79F3
:103CE000032B07D04BF2D410C0F200004FF0CB01F1
:103CF000FCF764FF009B9B79002B0BD0009B9B790A
:103D0000012B07D04BF2D410C0F200004FF0CC01D1
:103D1000FCF754FF009B1B79002B17D0009B1B79ED
:103D2000012B13D0009B1B79022B0FD0009B1B791A
:103D3000032B0BD0009B1B79042B07D04BF2D41024
:103D4000C0F200004FF0CD01FCF738FF019A4CF2B1
:103D50000003C4F200039A4205D14FF008004FF06F
:103D6000010101F03FFD019A40F20003C4F201039A
:103D70009A4205D14FF010004FF0010101F032FDE1
:103D8000019A48F20003C4F209039A4205D14FF0A8
:103D900080704FF0010101F025FD019A4CF2000303
:103DA000C4F209039A4205D14FF000704FF00101AF
:103DB00001F018FD019A40F20003C4F201039A4297
:103DC0004DD1019B4FF007021A72019B4FF0000288
:103DD0001A7203E0019B1B78DBB20393019B1B7DEE
:103DE000DBB203F00103DBB2002BF3D1019B6FF0D8
:103DF0007F0283F83020019B1B7DDBB203F02003A0
:103E0000002BF8D0019B4FF0000283F83020019B7B
:103E10004FF000025A60019B4FF000021A73019BA1
:103E20004FF000021A62019B4FF000021A74019BCE
:103E30004FF0000283F84C20019B4FF0000283F802
:103E40005420019B4FF0000283F85020019B1B7E01
:103E5000DBB20393019B1B7DDBB2039335E0019B37
:103E60004FF007021A72019B4FF000021A7203E032
:103E7000019B1B78DBB20393019B1B7DDBB203F03C
:103E80000103DBB2002BF3D1019B6FF07F0283F8BB
:103E90003020019B1B7DDBB203F02003002BF8D008
:103EA000019B4FF0000283F83020019B4FF000028D
:103EB0005A60019B4FF000021A73019B4FF0000201
:103EC0001A62019B1B7DDBB20393019A4CF2000343
:103ED000C4F209039A4204D1019B4FF0000283F817
:103EE0002420009B1B6801981946FFF739FD019AB1
:103EF00040F20003C4F201039A4206D1019B1B7BEE
:103F0000DBB203F0C003039305E0019B1B7BDBB234
:103F100003F0C0030393009B5B79012B04D0022BB9
:103F200007D0002B0FD009E0039B43F0010303935C
:103F30000AE0039B43F00203039305E0039B43F075
:103F40000303039300E000BF009B1B79002B23D0E9
:103F5000039B43F008030393009B1B7903F1FF339A
:103F6000032B19D801A252F823F000BF993F00009B
:103F70007D3F0000873F0000913F0000039B43F01E
:103F80001003039308E0039B43F02003039303E033
:103F9000039B43F030030393009B9B79012B03D1D8
:103FA000039B43F004030393019A40F20003C4F21D
:103FB00001039A4204D1019B039AD2B21A7303E01F
:103FC000039BDAB2019B1A7305B000BD00B583B044
:103FD0000190019A4CF20003C4F200039A421CD0F3
:103FE000019A40F20003C4F201039A4215D0019AEB
:103FF00048F20003C4F209039A420ED0019A4CF22F
:104000000003C4F209039A4207D04BF2D410C0F265
:1040100000004FF4CB71FCF7D1FD01984FF0000187
:1040200000F044FD019A4CF20003C4F200039A42EE
:1040300005D14FF008004FF0000101F0D3FB019AC9
:1040400040F20003C4F201039A4205D14FF0100080
:104050004FF0000101F0C6FB019A48F20003C4F2E0
:1040600009039A4205D14FF080704FF0000101F032
:10407000B9FB019A4CF20003C4F209039A4205D13C
:104080004FF000704FF0000101F0ACFB03B000BD39
:1040900082B00190019B4FF416521A60019B4FF0C1
:1040A00003025A71019B4FF000021A71019B4FF0FD
:1040B00000029A7102B0704700B583B001900B46C0
:1040C0008DF80330019A4CF20003C4F200039A42C7
:1040D0001CD0019A40F20003C4F201039A4215D0A9
:1040E000019A48F20003C4F209039A420ED0019AE1
:1040F0004CF20003C4F209039A4207D04BF2D410E9
:10410000C0F200004FF4ED71FCF758FD019A40F247
:104110000003C4F201039A4204D1019B9DF80320DD
:104120001A7003E0019B9DF803201A7003B000BDD4
:1041300000B583B00190019A4CF20003C4F2000371
:104140009A421CD0019A40F20003C4F201039A4241
:1041500015D0019A48F20003C4F209039A420ED026
:10416000019A4CF20003C4F209039A4207D04BF2C1
:10417000D410C0F2000040F2F311FCF71FFD019AC9
:1041800040F20003C4F201039A4203D1019B1B7861
:10419000DBB202E0019B1B78DBB2184603B000BD26
:1041A00000B58BB00390029101928DF80330029B11
:1041B0000993019B05939DF80330012B3ED14FF0ED
:1041C0000003069336E04FF0FF33079306E0079BAA
:1041D000002B0BD0079B03F1FF330793039B1B7D41
:1041E000DBB203F02003002BF1D000E000BF079BFF
:1041F000002B52D04FF01003089315E0099B1B7859
:10420000099A02F10102099203981946FFF754FF37
:10421000089B03F1FF330893059B03F1FF330593DC
:10422000069B03F101030693089B002B02D0059B1C
:10423000002BE3D1059B002BC5D131E04FF00003EB
:10424000069326E0039B1B7DDBB203F02003002BCB
:1042500025D04FF01003089315E0099B1B78099AAD
:1042600002F10102099203981946FFF725FF059B09
:1042700003F1FF330593089B03F1FF330893069B7B
:1042800003F101030693089B002B02D0059B002B32
:10429000E3D1059B002BD5D102E000BF00E000BFB9
:1042A000069B18460BB000BD00B589B00390029183
:1042B00001928DF80330029B0793019B04939DF8B4
:1042C0000330012B31D14FF00003059329E04FF06B
:1042D000FF33069306E0069B002B0BD0069B03F1F1
:1042E000FF330693039B1B7DDBB203F00103002B1E
:1042F000F1D000E000BF069B002B38D00398FFF7F9
:1043000017FF03461A46079B1A70079B03F1010328
:104310000793049B03F1FF330493059B03F101030F
:104320000593049B002BD2D124E04FF000030593AA
:1043300019E0039B1B7DDBB203F00103002B18D0B7
:104340000398FFF7F5FE03461A46079B1A70079B72
:1043500003F101030793059B03F101030593049BFC
:1043600003F1FF330493049B002BE2D102E000BF72
:1043700000E000BF059B184609B000BD00B583B042
:104380000190019A4CF20003C4F200039A421CD03F
:10439000019A40F20003C4F201039A4215D0019A37
:1043A00048F20003C4F209039A420ED0019A4CF27B
:1043B0000003C4F209039A4207D04BF2D410C0F2B2
:1043C000000040F28521FCF7F9FB019A40F200035E
:1043D000C4F201039A4208D1019B019A127BD2B226
:1043E00042F04002D2B21A7307E0019B1B7BDBB2A2
:1043F00043F04003DAB2019B1A7303B000BD00BF63
:1044000000B585B0019013460A468DF803208DF85B
:104410000230019A4CF20003C4F200039A421CD00D
:10442000019A40F20003C4F201039A4215D0019AA6
:1044300048F20003C4F209039A420ED0019A4CF2EA
:104440000003C4F209039A4207D04BF2D410C0F221
:1044500000004FF42B71FCF7B1FB9DF80230002BEC
:104460000BD09DF80230012B07D04BF2D410C0F2D4
:10447000000040F2AD21FCF7A1FB9DF80330062BB4
:104480002BD801A252F823F0A5440000AD4400004F
:10449000B5440000BD440000C5440000CD44000008
:1044A000D54400004FF00103039316E04FF00203E0
:1044B000039312E04FF0040303930EE04FF0080360
:1044C00003930AE04FF08003039306E04FF48073F8
:1044D000039302E04FF400730393019A40F2000348
:1044E000C4F201039A4224D19DF80330002B3CD042
:1044F0009DF80330012B38D09DF80330022B34D0C7
:104500009DF80330052B30D09DF80330062B2CD0BE
:104510009DF80330032B28D09DF80330042B24D0C2
:104520004BF2D410C0F2000040F2C921FCF746FB68
:104530001BE09DF80330002B17D09DF80330012BB2
:1045400013D09DF80330022B0FD09DF80330052BBC
:104550000BD09DF80330062B07D04BF2D410C0F2DD
:10456000000040F2CD21FCF729FB9DF80230012B21
:1045700016D1019A40F20003C4F201039A4207D116
:10458000019B019A5168039A41EA02025A602DE0A8
:10459000019B5A68039B42EA0302019B5A6025E093
:1045A000019A40F20003C4F201039A420FD1019A2A
:1045B000019B5968039B6FEA030301EA030140F280
:1045C0008F33C0F2000301EA030353600EE0019B46
:1045D0005A68039B6FEA030302EA030240F20733BF
:1045E000C0F2000302EA0303019A536005B000BD64
:1045F00000B583B00190019A4CF20003C4F20003AD
:104600009A421CD0019A40F20003C4F201039A427C
:1046100015D0019A48F20003C4F209039A420ED061
:10462000019A4CF20003C4F209039A4207D04BF2FC
:10463000D410C0F2000040F2FB21FCF7BFFA019A4F
:1046400040F20003C4F201039A4206D140F2000393
:10465000C4F201031B7DDBB202E0019B1B7DDBB2D8
:10466000184603B000BD00BF00B583B00190019AA9
:104670004CF20003C4F200039A421CD0019A40F2AB
:104680000003C4F201039A4215D0019A48F20003D4
:10469000C4F209039A420ED0019A4CF20003C4F20C
:1046A00009039A4207D04BF2D410C0F2000040F246
:1046B0001231FCF783FA019B9A6840F2CF33C0F2C3
:1046C000000302EA0303184603B000BD82B0019064
:1046D000019B1B7DDBB203F04003002B02D04FF0A7
:1046E000000301E04FF00103184602B0704700BF1D
:1046F00000B585B0019000914FF000038DF80F30A8
:10470000019A4CF20003C4F200039A421CD0019AB1
:1047100040F20003C4F201039A4215D0019A48F214
:104720000003C4F209039A420ED0019A4CF200032E
:10473000C4F209039A4207D04BF2D410C0F2000031
:104740004FF44E71FCF73AFA009BDB78002B13D044
:10475000009BDB78012B0FD0009BDB78022B0BD06A
:10476000009BDB78032B07D04BF2D410C0F2000083
:1047700040F23931FCF722FA009B9B78002B0BD0DA
:10478000009B9B78012B07D04BF2D410C0F20000A5
:1047900040F23A31FCF712FA009B1B78002B0BD049
:1047A000009B1B78012B07D04BF2D410C0F2000005
:1047B00040F23B31FCF702FA009B5B78002B0BD0F8
:1047C000009B5B78012B07D04BF2D410C0F20000A5
:1047D0004FF44F71FCF7F2F99DF80F3043F00103ED
:1047E0008DF80F30009BDB78012B04D0022B09D011
:1047F000002B19D00FE09DF80F3043F040038DF8E7
:104800000F3012E09DF80F306FEA43636FEA536395
:104810008DF80F3009E09DF80F306FEA83636FEA7F
:1048200093638DF80F3000E000BF009B5B78012B95
:1048300005D19DF80F3043F004038DF80F30009B35
:104840001B78012B05D19DF80F3043F002038DF842
:104850000F30009B9B78012B05D19DF80F3043F062
:1048600008038DF80F30019A40F20003C4F20103EF
:104870009A4206D1019A9DF80F3003F0CF031372CC
:1048800005E09DF80F3003F0CF03019A137205B0D5
:1048900000BD00BF82B00190019B4FF000029A70F2
:1048A000019B4FF00002DA70019B4FF001021A7079
:1048B000019B4FF001025A7002B0704700B587B0FB
:1048C0000390029113468DF80730039A4CF20003CF
:1048D000C4F200039A421CD0039A40F20003C4F2CF
:1048E00001039A4215D0039A48F20003C4F2090367
:1048F0009A420ED0039A4CF20003C4F209039A4282
:1049000007D04BF2D410C0F2000040F29331FCF714
:1049100055F99DF80730002B0BD09DF80730012B7F
:1049200007D04BF2D410C0F200004FF46571FCF7D1
:1049300045F94FF0000305939DF80730012B0FD187
:10494000029B1B78012B03D1059B43F002030593C7
:10495000029B5B78012B03D1059B43F00403059375
:10496000039A40F20003C4F201039A422BD19DF84E
:104970000730012B22D1039A039B1B7BDBB26FEA2A
:1049800043636FEA5363DBB21373039B4FF0000280
:104990001A70039B4FF000021A71039A039B1B7B52
:1049A000DBB203F07F031373039B4FF010029A6294
:1049B000039B059A42F001021A6230E0039B4FF01C
:1049C00000021A622BE09DF80730012B23D1039BD4
:1049D0001B7BDBB26FEA43636FEA5363DAB2039B7C
:1049E0001A73039B4FF000021A70039B4FF00002F2
:1049F0001A71039B1B7BDBB203F07F03039A1373D3
:104A0000039B4FF0100283F82820059B43F001021E
:104A1000039B1A6203E0039B4FF000021A6207B087
:104A200000BD00BF00B583B001900B46ADF8023069
:104A3000019A4CF20003C4F200039A421CD0019A7E
:104A400040F20003C4F201039A4215D0019A48F2E1
:104A50000003C4F209039A420ED0019A4CF20003FB
:104A6000C4F209039A4207D04BF2D410C0F20000FE
:104A70004FF47571FCF7A2F8019A40F20003C4F2FA
:104A800001039A4208D1019B1A6ABDF8023042EA3A
:104A90000302019B1A6207E0019B1A6ABDF802300B
:104AA00042EA0302019B1A6203B000BD00B583B065
:104AB00001900B468DF80330019A4CF20003C4F2CA
:104AC00000039A421CD0019A40F20003C4F2010391
:104AD0009A4215D0019A48F20003C4F209039A429F
:104AE0000ED0019A4CF20003C4F209039A4207D097
:104AF0004BF2D410C0F2000040F2EB31FCF75EF84C
:104B00009DF80330002B0BD09DF80330012B07D00C
:104B10004BF2D410C0F200004FF47B71FCF74EF85A
:104B20009DF80330012B20D1019A40F20003C4F21A
:104B300001039A420CD1019A019B93F83030DBB209
:104B40006FEA43636FEA5363DBB282F8303024E0EC
:104B5000019B93F83030DBB26FEA43636FEA536333
:104B6000DAB2019B83F8302017E0019A40F200038B
:104B7000C4F201039A4208D1019B93F83030019BA3
:104B80004FF0000283F8302007E0019B93F83030AB
:104B9000019B4FF0000283F8302003B000BD00BF3E
:104BA00000B583B001900B468DF80330019A4CF2AA
:104BB0000003C4F209039A4207D04BF2D410C0F2AA
:104BC000000040F21541FBF7F9FF9DF80330002B80
:104BD0000BD09DF80330012B07D04BF2D410C0F25C
:104BE000000040F21641FBF7E9FF9DF80330012B6E
:104BF0000AD1019B93F82430DBB243F00203DAB20E
:104C0000019B83F824200CE09DF80330002B08D191
:104C1000019B93F82430DBB203F03D03019A82F844
:104C2000243003B000BD00BF00B583B001900B4637
:104C30008DF80330019A4CF20003C4F209039A4242
:104C400007D04BF2D410C0F2000040F22D41FBF728
:104C5000B5FF9DF80330002B0BD09DF80330012BDE
:104C600007D04BF2D410C0F2000040F22E41FBF707
:104C7000A5FF9DF80330012B0AD1019B93F8243046
:104C8000DBB243F00103DAB2019B83F8242008E091
:104C9000019B93F82430DBB203F03E03019A82F8C3
:104CA000243003B000BD00BF00B585B001900B46B5
:104CB0008DF80330019A4CF20003C4F209039A42C2
:104CC00007D04BF2D410C0F2000040F24E41FBF787
:104CD00075FF9DF80330002B23D09DF80330012B86
:104CE0001FD09DF80330022B1BD09DF80330032BFF
:104CF00017D09DF80330042B13D09DF80330052BFB
:104D00000FD09DF80330062B0BD09DF80330072BF6
:104D100007D04BF2D410C0F2000040F24F41FBF735
:104D20004DFF9DF8033003F007034FEAC3030393DD
:104D3000019B93F82430DBB223F038030293039AEB
:104D4000029B42EA030343F004030293029BDBB29B
:104D500003F03F03019A82F8243005B000BD00BF84
:104D600000B585B0019013460A468DF803208DF8F2
:104D700002304FF000038DF80F30019A40F200032B
:104D8000C4F201039A4207D04BF2D410C0F20000E3
:104D900040F26E41FBF712FF9DF80330002B0BD061
:104DA0009DF80330012B07D04BF2D410C0F2000065
:104DB00040F26F41FBF702FF9DF80230002B0BD051
:104DC0009DF80230012B07D04BF2D410C0F2000046
:104DD0004FF48E61FBF7F2FE9DF80330002B02D0FA
:104DE000012B05D008E04FF001038DF80F3003E0F0
:104DF0004FF002038DF80F309DF80230012B0AD1DD
:104E0000019B1B7CDAB29DF80F3042EA0303DAB251
:104E1000019B1A7411E0019B1B7CDBB21A469DF8C2
:104E20000F306FEA0303DBB2DBB203F0F30302EAF5
:104E30000303DBB2DAB2019B1A7405B000BD00BFF8
:104E400000B585B0019013460A468DF803208DF811
:104E50000230019A40F20003C4F201039A4207D0E3
:104E60004BF2D410C0F2000040F29641FBF7A6FED0
:104E70009DF80330002B0FD09DF80330012B0BD091
:104E80009DF80330022B07D04BF2D410C0F2000083
:104E900040F29741FBF792FE9DF80230002B0BD0B9
:104EA0009DF80230012B07D04BF2D410C0F2000065
:104EB0004FF49361FBF782FE9DF80330012B08D07D
:104EC000022B0BD0002B0DD14FF010038DF80F30BB
:104ED00008E04FF040038DF80F3003E06FF07F03E0
:104EE0008DF80F309DF80230012B0AD1019B1B7CFD
:104EF000DAB29DF80F3042EA0303DAB2019B1A746A
:104F000011E0019B1B7CDBB21A469DF80F306FEA63
:104F10000303DBB2DBB203F0F30302EA0303DBB209
:104F2000DAB2019B1A7405B000BD00BF00B583B0B2
:104F30000190019A40F20003C4F201039A4207D0A3
:104F40004BF2D410C0F2000040F2C141FBF736FE34
:104F5000019B1B7EDBB2184603B000BD00B585B0D7
:104F600001900091019A40F20003C4F201039A42B9
:104F700007D04BF2D410C0F2000040F2D541FBF74D
:104F80001DFE009B9B78002B0BD0009B9B78012B78
:104F900007D04BF2D410C0F2000040F2D641FBF72C
:104FA0000DFE009BDB78002B0BD0009BDB78012BE8
:104FB00007D04BF2D410C0F2000040F2D741FBF70B
:104FC000FDFD009BDB79FF2B07D14BF2D410C0F223
:104FD00000004FF49B61FBF7F1FD009B5B79002B18
:104FE0000BD0009B5B79012B07D04BF2D410C0F2A1
:104FF000000040F2D941FBF7E1FD009B1B79002B3B
:105000000BD0009B1B79012B07D04BF2D410C0F2C0
:10501000000040F2DA41FBF7D1FD009B9B79FF2BAA
:1050200007D14BF2D410C0F2000040F2DB41FBF795
:10503000C5FD009B1B78002B0BD0009B1B78012B20
:1050400007D04BF2D410C0F2000040F2DC41FBF775
:10505000B5FD009B5B78002B0BD0009B5B78012B90
:1050600007D04BF2D410C0F2000040F2DD41FBF754
:10507000A5FD4FF000030393009BDB78012B18D1B3
:10508000039B43F010030393009B5B79012B03D137
:10509000039B43F020030393009B1B79012B03D157
:1050A000039B43F008030393009BDA79019B83F889
:1050B0005420009B1B78012B03D1039B43F0010379
:1050C0000393009B9B78012B08D1039B43F00403BF
:1050D0000393009B9A79019B83F85020009B5B7897
:1050E000002B03D1039B43F002030393039BDBB22A
:1050F00003F03F03019A82F84C30019B1B7BDBB22B
:1051000043F03803DAB2019B1A7305B000BD00BF4B
:1051100082B001900B468DF803309DF80330012BCF
:1051200009D1019B93F84C30DBB203F0FD03019AE7
:1051300082F84C3009E0019B93F84C30DBB243F02D
:105140000203DAB2019B83F84C2002B0704700BF23
:1051500000B587B00390029101928DF803309DF85D
:105160000330002B27D0039B1B7B8DF812309DF85A
:1051700012308DF813309DF8123023F010038DF8A3
:105180001230039B9DF812201A73039B1846029954
:10519000019A4FF00103FFF703F803460593039BC1
:1051A0001B7DDBB203F04003002BF8D0039B9DF87E
:1051B00013201A7310E0039B18460299019A4FF0CE
:1051C0000103FEF7EDFF03460593039B1B7DDBB256
:1051D00003F04003002BF8D0059B184607B000BD34
:1051E00000B583B001900B468DF803300DF1030339
:1051F000019819464FF001024FF00103FFF7A8FF95
:1052000003B000BD00B585B00390029101920398F0
:105210000299019A4FF00003FFF79AFF03461846E0
:1052200005B000BD4CF20003C4F20F03D3F8883080
:105230004FEA136303F00303032B40F0AA804CF200
:105240000003C4F20F03D3F80C3103F00303032B64
:1052500000F2F48001A252F823F000BF6D5200006A
:10526000D1520000375300006D5200004CF2000391
:10527000C4F20F03D3F888304FEA43434FEA534355
:1052800003F1010241F20023C0F27A0303FB02F2B0
:105290004CF20003C4F20F03D3F888304FEA1343F3
:1052A00003F0FF0303F10103B2FBF3F24CF200033E
:1052B000C4F20F03D3F8043103F0FF0303F1010339
:1052C000B2FBF3F240F21C03C1F200031A60B6E035
:1052D0004CF20003C4F20F03D3F888304FEA434383
:1052E0004FEA534303F1010243F20063C0F26E132D
:1052F00003FB02F24CF20003C4F20F03D3F8883030
:105300004FEA134303F0FF0303F10103B2FBF3F28F
:105310004CF20003C4F20F03D3F8043103F0FF038F
:1053200003F10103B2FBF3F240F21C03C1F20003EC
:105330001A6000BF83E04CF20003C4F20F03D3F8FD
:1053400088304FEA43434FEA534303F101034FEAE6
:1053500003424CF20003C4F20F03D3F888304FEA43
:10536000134303F0FF0303F10103B2FBF3F24CF22A
:105370000003C4F20F03D3F8043103F0FF0303F179
:105380000103B2FBF3F240F21C03C1F200031A6006
:1053900055E04CF20003C4F20F03D3F80C3103F0D4
:1053A0000303032B4BD801A252F823F0BD53000096
:1053B000E953000015540000BD5300004CF20003F7
:1053C000C4F20F03D3F8043103F0FF0303F1010229
:1053D00040F60013C0F23D03B3FBF2F240F21C03AF
:1053E000C1F200031A602AE04CF20003C4F20F037A
:1053F000D3F8043103F0FF0303F1010241F6003357
:10540000C0F2B703B3FBF2F240F21C03C1F2000397
:105410001A6014E04CF20003C4F20F03D3F8043115
:1054200003F0FF0303F101034FF40042B2FBF3F278
:1054300040F21C03C1F200031A6000E000BF704795
:105440004CF20003C4F20F034FF02002C3F8A02176
:105450004CF20003C4F20F03D3F8A03103F0200391
:10546000002B09D04CF20003C4F20F03D3F8A03193
:1054700003F04003002BF5D04CF20003C4F20F03FD
:105480004FF00302C3F804214CF20003C4F20F03EF
:105490004FF00002C3F8A8214CF20003C4F20F033E
:1054A0004FF00002C3F8AC214CF20003C4F20F032A
:1054B0004FF00102C3F80C214CF20003C4F20F03B9
:1054C00040F26302C0F20502C3F884204CF20003EC
:1054D000C4F20F034FF0AA02C3F88C204CF2000371
:1054E000C4F20F034FF05502C3F88C204CF20003B6
:1054F000C4F20F034FF00102C3F880204CF2000306
:10550000C4F20F034FF0AA02C3F88C204CF2000340
:10551000C4F20F034FF05502C3F88C204CF2000385
:10552000C4F20F03D3F8883003F08063002BF5D06A
:105530004CF20003C4F20F034FF00302C3F88020C3
:105540004CF20003C4F20F034FF0AA02C3F88C2000
:105550004CF20003C4F20F034FF05502C3F88C2045
:105560004CF20003C4F20F03D3F8883003F0407309
:10557000002BF5D04CF20003C4F20F034FF02302CE
:10558000C3F8A4204CF20003C4F20F034FF0AA02A8
:10559000C3F8AC204CF20003C4F20F034FF05502E5
:1055A000C3F8AC204CF20003C4F20F034FF0010229
:1055B000C3F8A0204CF20003C4F20F034FF0AA027C
:1055C000C3F8AC204CF20003C4F20F034FF05502B5
:1055D000C3F8AC204CF20003C4F20F03D3F8A83098
:1055E00003F48063002BF5D04CF20003C4F20F03E8
:1055F0004FF00302C3F8A0204CF20003C4F20F03E3
:105600004FF0AA02C3F8AC204CF20003C4F20F031F
:105610004FF05502C3F8AC204CF20003C4F20F0364
:10562000D3F8A83003F44073002BF5D04CF20003FC
:10563000C4F20F0348F2DE72C0F22842C3F8C4205D
:105640004CF20003C4F20F034FF00002C3F8C8216C
:105650004CF20003C4F20F0343F23A021A604EF612
:105660000053CEF200034FF000029A60704700BF73
:1056700084B001900091019B1F2B03D9019BA3F1E2
:10568000200300E0019B0393019B1F2B27D84CF2C2
:105690000003C4F20F034CF20002C4F20F02D2F86E
:1056A000A811039A4FF0030000FA02F26FEA020217
:1056B00001EA0202C3F8A8214CF20003C4F20F036E
:1056C0004CF20002C4F20F02D2F8A811039A00981B
:1056D00000FA02F241EA0202C3F8A82126E04CF2E5
:1056E0000003C4F20F034CF20002C4F20F02D2F81E
:1056F000AC11039A4FF0030000FA02F26FEA0202C3
:1057000001EA0202C3F8AC214CF20003C4F20F0319
:105710004CF20002C4F20F02D2F8AC11039A0098C6
:1057200000FA02F241EA0202C3F8AC2104B0704769
:1057300084B00190019B1F2B09D8019B02934CF26E
:105740000003C4F20F03D3F8A83103930AE0019BCE
:10575000A3F1200302934CF20003C4F20F03D3F829
:10576000AC310393029B039A22FA03F303F0030381
:105770000393039B184604B0704700BF00B585B083
:10578000019040F21C03C1F200031B6802930198D0
:10579000FFF7CEFF03460393039B032B19D801A207
:1057A00052F823F0B5570000BD570000C557000060
:1057B000CD5700004FF0040303930AE04FF00103BC
:1057C000039306E04FF00203039302E04FF0080357
:1057D0000393029A039BB2FBF3F30293029B1846D6
:1057E00005B000BD82B001900B468DF803309DF8E6
:1057F0000330012B15D14CF20002C4F20F024CF21F
:105800000003C4F20F03D3F8C41001984FF2DE7303
:10581000CEF6EF7300EA030341EA0303C2F8C43093
:105820001AE09DF80330002B16D14CF20002C4F2AE
:105830000F024CF20003C4F20F03D3F8C410019B13
:105840006FEA030301EA03014FF2DE73CEF6EF7352
:1058500001EA0303C2F8C43002B070474CF20003FF
:10586000C4F20F034FF00002C3F8C02030BF7047EE
:105870004EF60053CEF200034FF004021A614CF2D0
:105880000003C4F20F034FF00802C3F8C02030BF7A
:10589000704700BF4EF60053CEF200034FF00402F3
:1058A0001A614CF20003C4F20F034FF00902C3F86F
:1058B000C02030BF704700BF4EF60053CEF2000349
:1058C0004FF004021A614CF20003C4F20F034FF0D0
:1058D0000302C3F8C02030BF704700BF4BB942B9C4
:1058E000002908BF002802D04FF0FF31084600F021
:1058F00037B882B0EC462DE9005000F005F8DDF82D
:1059000004E002B00CBC7047F8B514461D460646CC
:105910000F4600F0D9F900FB05F5A0FB042304FBBA
:105920000154E318B61A67EB0307069BC3E9006747
:10593000F8BD00BFF8B514461D4606460F4600F0F8
:1059400011F800FB05F5A0FB042304FB0154E31848
:10595000B61A67EB0307069BC3E90067F8BD00BFF3
:10596000704700BF00292DE9F04F85B0C0F2C88014
:105970000026002BC0F2BF808946144605469B4690
:10598000002B4AD18A4257D9B2FA82F353B1C3F1FC
:10599000200001FA03F925FA00F812FA03F49D40F9
:1059A00048EA0909270C484639461FFA84FB00F0EB
:1059B0000BFB39468246484600F034FC2A0C0BFBB0
:1059C0000AF342EA01494B4509D919EB04090AF1E6
:1059D000FF3A04D24B4584BF0AF1FF3AA144C3EB1E
:1059E000090939464846ADB200F0EEFA394680461C
:1059F000484600F017FC0BFB08FB45EA0145AB45A8
:105A000007D92D1908F1FF3803D2AB4588BF08F13B
:105A1000FF3848EA0A48002703E08B4257D900279D
:105A2000B84642463B4616B1524263EB4303194621
:105A3000104605B0BDE8F08F22B91146012000F0F4
:105A4000C3FA0446B4FA84F8B8F1000F5ED1C4EB8F
:105A50000908270C1FFA84F90121029139464046B2
:105A600000F0B2FA39468246404600F0DBFB4FEACE
:105A7000154809FB0AF348EA014B5B4509D91BEBC2
:105A8000040B0AF1FF3A04D25B4584BF0AF1FF3AE6
:105A9000A344C3EB0B0B39465846ADB200F094FA61
:105AA00039468046584600F0BDFB09FB08F945EA37
:105AB0000145A94507D92D1908F1FF3803D2A94599
:105AC00088BF08F1FF3848EA0A48029FA9E7B3FAFD
:105AD00083F7002F68D18B422CBF4FF000094FF0A5
:105AE000010982428CBF4C4649F00104002C96D03B
:105AF0004FF0010895E7524263EB4303F6433BE75F
:105B0000404261EB41014FF0FF3632E704FA08F4FE
:105B1000C8F1200735FA07F329FA07FA270C09FA22
:105B200008FB3946504643EA0B02029200F04CFA59
:105B300039461FFA84F98346504600F073FB0298F9
:105B400009FB0BF2030C43EA01439A4204D91B19E7
:105B50000BF1FF3BC0F0B1809B1A39461846019308
:105B600000F032FA019982460846394600F05AFBA5
:105B7000DDF808C009FB0AF31FFA8CF040EA014285
:105B8000934208D912190AF1FF3A04D2934284BF12
:105B90000AF1FF3A121905FA08F54AEA0B4EC3EB6F
:105BA0000208CDF808E059E7C7F1200003FA07FA28
:105BB000C24035FA00F342EA0A0B21FA00F801FA72
:105BC00007F940464FEA1B4A43EA09010291514650
:105BD0001FFA8BF2039200F0F7F9514681464046D6
:105BE00000F020FB039BDDF808C003FB09F24FEA3D
:105BF0001C4014FA07F340EA0144A24204D914EB12
:105C00000B0409F1FF3952D3A41A514620460193DF
:105C100000F0DAF951468046204600F003FB039875
:105C2000DDF808C000FB08F21FFA8CF343EA0140DC
:105C3000019B824204D910EB0B0008F1FF3830D3EE
:105C400048EA09481FFA83FC1B0C801A1FFA88FED9
:105C50004FEA184A0CFB0EF90CFB0AFC03FB0EC1C1
:105C600003FB0AF201EB19418C4588BF02F5803233
:105C700002EB114E704510D31FFA89F905FA07F7A8
:105C800009EB014014BF0022012287422CBF0027EC
:105C900002F00107002F3FF4C4AE08F1FF380027DF
:105CA000BFE6824284BF584408F1FF38C8E7A242E9
:105CB00084BF09F1FF395C44A6E79A4284BF0BF127
:105CC000FF3B1B1948E700BF2DE9F04F0C4683B09E
:105CD0008046164689461F4615468A46002B4BD1FC
:105CE0008A425CD9B2FA82F35BB1C3F1200001FAB7
:105CF00003FA28FA00F216FA03F508FA03F842EA62
:105D00000A0A2E0C50463146AFB200F05DF931461A
:105D10004FEA18448146504600F084FA07FB09F325
:105D200044EA014A534509D91AEB050A09F1FF393A
:105D300004D2534584BF09F1FF39AA44C3EB0A0AD0
:105D4000314650461FFA88F800F03EF931460446C5
:105D5000504600F067FA07FB04F748EA0148474558
:105D600006D9013C18EB050802D2474588BF013C23
:105D700044EA094400265CE08B4258D8B3FA83F623
:105D8000002E5BD18B422CBF0022012285428CBFAA
:105D9000154642F00105002D49D0012449E022B901
:105DA0001146012000F010F90546B5FA85F6002EDF
:105DB00040F0BA80641B2F0C1FFA85FA0126394681
:105DC000204600F001F939464FEA184B814620463B
:105DD00000F028FA0AFB09F34BEA014B5B4509D9AD
:105DE0001BEB050B09F1FF3904D25B4584BF09F1B8
:105DF000FF39AB44C3EB0B0B394658461FFA88F802
:105E000000F0E2F839460446584600F00BFA0AFB67
:105E100004FA48EA0148C24506D9013C18EB0508D6
:105E200002D2C24588BF013C44EA094401E0002691
:105E300034463146204603B0BDE8F08FC6F120005D
:105E4000B34032FA00F721FA00FB1F4314FA06F2BE
:105E500028FA00F158464FEA174A1143009151467B
:105E6000BBB2019300F0B0F85146B54081465846A8
:105E700000F0D8F9019C009804FB09F34FEA104C9C
:105E80004CEA014B5B4505D91BEB070B09F1FF39C8
:105E9000C0F08E80C3EB0B0B5146584600F094F8CF
:105EA00051460446584600F0BDF90198009A00FB9F
:105EB00004F31FFA82FC4CEA0142934206D9013CEA
:105EC000D21903D2934201D9D219013C44EA0944C0
:105ED000A8B2D21A2D0C1FFA84FC230C00FB0CF77D
:105EE00000FB03FE05FB0CE105FB03F501EB17418D
:105EF0008E4588BF05F5803505EB1145AA4210D3C4
:105F0000BFB208FA06F607EB014214BF4FF0000ECD
:105F10004FF0010E96422CBF00260EF00106002E17
:105F200087D0013C002684E7B540C6F1200124FA61
:105F300001F928FA01F22F0CB440394648462243B1
:105F4000009200F041F839461FFA85FA8346484628
:105F500000F068F9009B1A0C0AFB0BF342EA0144BB
:105F6000A34203D964190BF1FF3B27D3E41A394646
:105F7000204600F029F839468146204600F052F9C3
:105F800000980AFB09F31FFA80FC4CEA0144A34283
:105F900008D9641909F1FF3904D2A34284BF09F179
:105FA000FF39641908FA06F8E41A49EA0B4606E7CD
:105FB0005B4584BF09F1FF39BB446BE7A34284BF53
:105FC0000BF1FF3B6419D1E74A1E08BF7047C0F0D0
:105FD0002481884240F21681114200F01781B0FA04
:105FE00080F3B1FA81F2A2EB0303C3F11F0304A211
:105FF00002EB03134FF000029F4600BFAFF3008097
:10600000B0EBC17F00BF42EB020228BFA0EBC17022
:10601000B0EB817F00BF42EB020228BFA0EB817092
:10602000B0EB417F00BF42EB020228BFA0EB417002
:10603000B0EB017F00BF42EB020228BFA0EB017072
:10604000B0EBC16F00BF42EB020228BFA0EBC16002
:10605000B0EB816F00BF42EB020228BFA0EB816072
:10606000B0EB416F00BF42EB020228BFA0EB4160E2
:10607000B0EB016F00BF42EB020228BFA0EB016052
:10608000B0EBC15F00BF42EB020228BFA0EBC150E2
:10609000B0EB815F00BF42EB020228BFA0EB815052
:1060A000B0EB415F00BF42EB020228BFA0EB4150C2
:1060B000B0EB015F00BF42EB020228BFA0EB015032
:1060C000B0EBC14F00BF42EB020228BFA0EBC140C2
:1060D000B0EB814F00BF42EB020228BFA0EB814032
:1060E000B0EB414F00BF42EB020228BFA0EB4140A2
:1060F000B0EB014F00BF42EB020228BFA0EB014012
:10610000B0EBC13F00BF42EB020228BFA0EBC130A1
:10611000B0EB813F00BF42EB020228BFA0EB813011
:10612000B0EB413F00BF42EB020228BFA0EB413081
:10613000B0EB013F00BF42EB020228BFA0EB0130F1
:10614000B0EBC12F00BF42EB020228BFA0EBC12081
:10615000B0EB812F00BF42EB020228BFA0EB8120F1
:10616000B0EB412F00BF42EB020228BFA0EB412061
:10617000B0EB012F00BF42EB020228BFA0EB0120D1
:10618000B0EBC11F00BF42EB020228BFA0EBC11061
:10619000B0EB811F00BF42EB020228BFA0EB8110D1
:1061A000B0EB411F00BF42EB020228BFA0EB411041
:1061B000B0EB011F00BF42EB020228BFA0EB0110B1
:1061C000B0EBC10F00BF42EB020228BFA0EBC10041
:1061D000B0EB810F00BF42EB020228BFA0EB8100B1
:1061E000B0EB410F00BF42EB020228BFA0EB410021
:1061F000B0EB010F00BF42EB020228BFA0EB010091
:10620000104670470CBF012000207047B1FA81F2A0
:10621000C2F11F0220FA02F0704708B14FF0FF30C0
:10622000FFF79EBB0029F8D02DE90340FFF7CCFE15
:10623000BDE8064002FB00F3A1EB0301704700BF7D
:1062400070B5044688B104F1480253685D1E07D456
:10625000023302EB830656F8043D9847013DFAD518
:10626000A36A0BB12046984770BD40F22003C1F2EB
:1062700000031C68E7E700BF70B50C4609680546D7
:1062800009B1FFF7F9FF28462146BDE8704002F04A
:10629000ABBB00BF40F22003C1F2000370B51B6826
:1062A0000546984246D0436A1946BBB1DA68AAB19E
:1062B0000026915941B10C68284602F095FB214611
:1062C000002CF8D16B6ADA6804363C2E01D0DA680B
:1062D000EFE71146284602F087FB696A096811B1A9
:1062E000284602F081FB696911B1284602F07CFB67
:1062F000696A11B1284602F077FBA96B11B12846F3
:1063000002F072FBE96B11B1284602F06DFB296CBB
:1063100011B1284602F068FBAB6CD3F8881011B1BC
:10632000284602F061FB696B11B1284602F05CFB64
:10633000AB6903B970BDAB6A28469847D5F8D81049
:106340000029F7D02846BDE8704095E70EB440F22A
:10635000200330B59CB01FACC1F20003054601A973
:1063600054F8042B4FF0FF3C18684FF40273ADF85B
:1063700010302346059501956FF00045ADF812C029
:10638000069503951B9400F0B9F8019B00221A7042
:106390001CB0BDE8304003B0704700BF0CB40B46E2
:1063A00010B59CB01EAC01A905934FF4027C54F8C3
:1063B000042B01934FF0FF33ADF8123023461B94AA
:1063C0006FF00044ADF810C00694039400F096F806
:1063D000019B00221A701CB0BDE8104002B070474B
:1063E0002DE9F04F85B092460C46039090681768EF
:1063F000002800F081804FF000090B684D46002D09
:1064000054D0A668B542B0463EBF18462E46A846B0
:106410003CD3A08910F4906F08BF184636D062694B
:10642000216902EB420B5B1A03F1010C0BEBDB7BE6
:10643000AC444FEA6B0BE3455A463CBFE3465A4631
:1064400010F4806F37D011460398019302F0F6FBE9
:10645000019B00283BD01A4621690193029002F06B
:10646000F9FEA289019BDDF808C022F4906242F097
:106470008002A2812E46A846C3EB0B020CEB030060
:10648000A260C4F810C02060C4F814B04246494667
:1064900002F0A8FFA2682368961BA660DAF808201D
:1064A00043442360551BCAF80850FDB1D7F800904B
:1064B0007D680837A3E70398019303F09FFC019BD5
:1064C00084460028D6D10398216902F08DFA039AF8
:1064D0000C234FF0FF3013600023A289CAF8043068
:1064E00042F04002CAF80830A28102E02846CAF809
:1064F000045005B0BDE8F08F5060FAE72DE9F04F89
:10650000C5B00E469A461546099002F053FBB38972
:1065100013F0800F00681B9003D03369002B01F04B
:106520008C800DF17409B3464C4600221092002372
:10653000189217921A920D922DAA199328320DF1E2
:10654000F703169207930023CDF8DC903893399324
:106550002B78B3F1250218BF0122002B0CBF0022BB
:1065600002F0010202B32E4616F8013F1A1E18BFB0
:106570000122252B0CBF002202F00102002AF3D1D8
:10658000771B08BF35460FD06760389B399A0133B7
:106590002560D219072B3992389379DC08340D988D
:1065A0003546C0190D903378002B00F03787002155
:1065B0004FF00002CDF828A06B1C0C914FF0FF3873
:1065C0008DF80F218A466A782B204FF0200C5D1C35
:1065D000A2F12003582B00F21982DFE813F0290200
:1065E00017021702350217021702170217021702C5
:1065F00017023C0248021702C802CF021702EF023C
:10660000F602F602F602F602F602F602F602F602CA
:10661000F6021702170217021702170217021702D3
:106620001702170217024F02880217028802170288
:10663000170217021702C10217021702EE03170210
:106640001702170217021702930317021702AD036E
:106650001702170217021702170217021702170272
:1066600017021702C703D8038802880288020B03A7
:10667000D803170217020F031702190329033E0359
:106680008C03170259031702840317021702EA004A
:106690000998594637AAFFF7A3FE00287CD14C463B
:1066A0007DE71899012940F35284119A0123636010
:1066B000389B2260399A013338930132072B399283
:1066C00000F39685083401236360389B399A0133BF
:1066D0001B980132072B39922060389300F37D8597
:1066E0000834109800220023199904F06BFB00284D
:1066F00040F003851899119B4A1E6260591C389B13
:1067000021603999013338938A18072B399200F3A5
:106710002F8408341A9A1A9862603EAA389B226025
:10672000399A013338931218072B399200F34F81AD
:1067300004F108031AF0040F00F056810C990B9A2B
:106740008E1A002E40F35081102E4BF2E417D8BF62
:10675000C0F2000740F3DE831024C0F200070DF101
:10676000DC08DDF824A003E0103E102E40F3D283B5
:106770005C60389A399901321F601031072A3991CB
:1067800003F108033892EFDD504659464246FFF7C1
:1067900027FE4B460028E7D05E46B3890D9813F0DC
:1067A000400F18BF4FF0FF300D900D9845B0BDE879
:1067B000F08F1AF0200F4BF22820C0F20000149244
:1067C000179000F0C3820A99CB1D23F0070303F151
:1067D00008020A92D3E9006756EA07010CBF0022BB
:1067E00001221AEA020F40F0BC8402234FF000019C
:1067F0008DF80F11B8F1000FA8BF2AF0800AB8F188
:10680000000F18BF42F00102002A00F06081012B46
:1068100000F03484022B00F017841699CDF82C80F8
:1068200011914FEAD6084FEAD70C48EA477806F0AC
:10683000070067464646303056EA070201F8010D68
:10684000EFD11AF0010FDDF82C80119140F0DB84BC
:10685000169B5B1A0E930E9BCDF854804345B8BF30
:1068600043460B939DF80F3113B10B9901310B91F6
:106870001AF00202139202D00B9B02330B931AF010
:106880008400129038D10C990B9A8E1A002E33DDA9
:10689000102E4BF2E417D8BFC0F2000720DD4FF0F6
:1068A0001008C0F2000702E0103E102E18DDC4F8F8
:1068B0000480389B399A013327601032072B3992B4
:1068C00004F108043893EFDD0998594637AA4C467D
:1068D000FFF786FD00287FF45FAF103E102EE6DC48
:1068E0006660389B27605A1C399B38929B19072A8F
:1068F000399300F3F78308349DF80F3173B1012306
:106900006360389B43AA03322260399A013338937B
:106910000132072B399200F340830834139B6BB18B
:1069200002236360389B43AA2260399A013338936B
:106930000232072B399200F33A83083412988028E8
:1069400000F0B28215980E9BC61A002E2EDD102E76
:10695000A74FC8BF4FF0100803DC1BE0103E102EFD
:1069600018DDC4F80480389B399A0133276010324F
:10697000072B399204F108043893EFDD0998594642
:1069800037AA4C46FFF72CFD00287FF405AF103ED8
:10699000102EE6DC6660389B27605A1C399B3892C3
:1069A0009B19072A399300F3EE8208341AF4807F8A
:1069B00040F019820E99119A6160389B2260399AD1
:1069C000013338935218072B39927FF7B1AE0998EB
:1069D000594637AAFFF704FD00287FF4DDAE1AF010
:1069E000040F4B467FF4AAAE399B0D980B9A0C9975
:1069F0008A42ACBF801840180D90002B40F09E8258
:106A00000023DDF828A038934C46A1E51492002A13
:106A100000F0048501208DF8B4204FF000012DAA6C
:106A20000B908DF80F1111920E90002115911FE718
:106A30009DF80F31002B40F00C840A992B468DF8FD
:106A40000FC12A780A91C2E50A994AF0010A2A7808
:106A50002B460A91BBE50A9B0A9A1B68111D002B65
:106A60000C93C0F2B2852A782B460A91AFE50A99B9
:106A70002B468DF80F012A780A91A8E54AF0100AF2
:106A800014921AF0200F00F087810A98C31D23F09A
:106A9000070303F108010A91D3E90067002E77F19B
:106AA0000000C0F2768356EA07014FF001030CBFE5
:106AB00000220122B8F1000FA8BF2AF0800AB8F125
:106AC000000F18BF42F00102002A7FF4A0AE002B95
:106AD00040F0E5811AF0010F00F0E18130238DF8DC
:106AE000DB302DAB012027330E901193B3E61AF063
:106AF000080F149200F0BF830A98C31D23F0070308
:106B000003F108010A915E681F68199610973846CC
:106B1000314603F04DFB0346002800F093843846CD
:106B200000220023314604F057F9002840F0158474
:106B30009DF80F3103204BF21C224BF218210B90D1
:106B40001498C0F20001C0F200022AF0800A47281F
:106B5000D8BF0A460321119200220E91159283E6B6
:106B60000A994AF0080A2A782B460A912FE50A99D1
:106B70002A784AF0040A2B460A9128E52B4613F896
:106B8000012B2A2A00F0CF86A2F13001092988BF03
:106B90004FF0000810D802354FF0000815F8012C0E
:106BA00008EB88082B46013501EB4808A2F13001BB
:106BB0000929F3D948EAE8781D4609E50A994AF017
:106BC000800A2A782B460A9101E5A2F130010026BD
:106BD0002B4606EB860613F8012B01EB4606A2F1C5
:106BE00030011D460929F3D90C961D46F0E400BF7B
:106BF000F4B100004AF0400A0A9934E72A786C2A76
:106C000000F018840A994AF0100A2B460A91DEE433
:106C10001AF0200F00F023830A990D9A0B68104692
:106C20004FEAE0710A9AC3E9000102F1040A8FE415
:106C30001AF02003149200F0C7800A9BDA1D00238B
:106C400022F0070202F108000A90D2E9006756EA32
:106C500007010CBF00220122C8E50A9A4BF2282046
:106C60000A997823C0F200001493166804318DF855
:106C70000D314AF0020A3023321E18BF01228DF86E
:106C80000C3136464FF00007179002230A91ADE50C
:106C90000A9B14924FF00002181D8DF80F211B68FB
:106CA0000A901193002B00F04D85B8F1000F119858
:106CB000C0F22A850021424602F092FA03460028DB
:106CC00000F06E8511981B1A0E93434540F38284A1
:106CD000CDF83880002128EAE8789DF80F31CDF80A
:106CE0002C801591C0E51AF0200F149210D00A9B49
:106CF000DA1D0123A4E70A994AF0200A2A782B46D4
:106D00000A9164E44AF0100A14921AF0200FEED1AE
:106D10001AF0100F40F054821AF0400F00F0508229
:106D20000A980123011D0A910688321E18BF01220C
:106D300036464FF0000759E51AF0200F14924BF237
:106D40000422C0F2000217927FF43DAD1AF0100F3A
:106D500040F02D821AF0400F00F029820A990A1D96
:106D60000A920E8836464FF0000735E5149201204E
:106D70000A9A4FF000010B900E90136804328DF8C0
:106D80000F110A922DAA8DF8B43011924DE61AF027
:106D9000200F14927FF479AE1AF0100F40F0ED81BD
:106DA0001AF0400F00F0E9810A98011D0A91B0F92C
:106DB000006036464FEAE67770E64AF0100A149211
:106DC0001AF020037FF439AF1AF0100200F05F824E
:106DD0000A9A101D0A901668321E18BF0122364604
:106DE0004FF0000702E5149B652B7FF75AAC109813
:106DF00000220023199903F0E5FF002800F0E1804C
:106E000001236360389A4BF24423C0F200032360ED
:106E1000399B013238920133072A3993D8BF04F1E4
:106E2000080300F39F82429A1898824203DB1AF00B
:106E3000010F3FF47FAC1B9901225A60389A196008
:106E40003999013238920131072A399100F3EB83E5
:106E50000833189A561E002E7FF76CAC102EA04FE8
:106E600040F3E98110240DF1DC0803E0103E102E00
:106E700040F3E1815C60389A399901321F6010312A
:106E8000072A399103F108033892EFDD0998594632
:106E90004246FFF7A5FA4B460028E7D07CE4169956
:106EA00000220E921191D6E40C990B9A8E1A002EA4
:106EB0007FF748AD102E8A4FC8BF4FF0100803DC93
:106EC0001BE0103E102E18DDC4F80480389B399A60
:106ED000013327601032072B399204F108043893EC
:106EE000EFDD0998594637AA4C46FFF779FA002892
:106EF0007FF452AC103E102EE6DC6660389B2760B3
:106F00005A1C399B38929B19072A399300F38881C0
:106F1000083417E55E60389A1F60399B0132389259
:106F2000F318072A39937FF760AD0998594637AAB5
:106F3000FFF756FA00283FF457AD2DE4099859465B
:106F400037AAFFF74DFA00283FF45AAD24E41AF0AF
:106F5000010F7FF4AAAB01236360389B399A013398
:106F600011990132072B3992216038937FF7D1AB09
:106F70000998594637AAFFF733FA00287FF40CAC7A
:106F80004C46FFF7C7BB0998594637AAFFF728FABE
:106F900000287FF401AC4C4608E50998594637AA09
:106FA000FFF71EFA00287FF4F7AB4C46B6E40998C9
:106FB000594637AAFFF714FA00287FF4EDAB4C4688
:106FC000BCE4429B002B40F3D98118998B42C0F25C
:106FD0006F81119A6160389B2260399A013338932E
:106FE0005218072B3992D8BF04F1080300F3BA8373
:106FF000429C1898241A002C40F39B81102C384F87
:1070000040F38B81CDF838A01026AA460DF1DC089C
:10701000099D03E0103C102C40F37C815E60389A9F
:10702000399901321F601031072A399103F10803A1
:107030003892EFDD284659464246FFF7D1F94B46D4
:107040000028E7D0FFF7A8BB1698DDF85CC0034620
:107050001190310906F00F0241EA077138091CF856
:1070600002200E46074656EA070103F8012DF0D12B
:10707000169A1193D21A0E92FFF7EDBB0023092244
:10708000B24273EB0700169B3EBFCDF82C80A046A2
:107090001C461AD2304639460A220023FEF71EFC4F
:1070A00030463946002302F1300C0A2204F801CDA3
:1070B000FEF714FC06460F4609200021B042B941F4
:1070C000E8D323464446DDF82C805A1E3036119210
:1070D00003F8016C169B9B1A0E93FFF7BCBB00BF15
:1070E000F4B100000998594637AAFFF779F900284A
:1070F0007FF452AB4C46FFF7FFBB1898461E002E9C
:107100007FF708AB102E9C4FC8BF4FF0100803DC70
:107110001BE0103E102E18DDC4F80480389B399A0D
:10712000013327601032072B399204F10804389399
:10713000EFDD0998594637AA4C46FFF751F9002868
:107140007FF42AAB103E102EE6DC6660389B399A3D
:10715000013327609219072B399238937FF7D9AA08
:1071600006E7149830214AF0020A012202238DF822
:107170000C118DF80D01FFF739BB0A9A131D166823
:107180000A9336464FEAE677002E77F10000BFF605
:107190008AAC764267EB47072D2356EA07028DF843
:1071A0000F310CBF002201220123FFF723BB0A9BF2
:1071B000181D1E680A9036464FF00007FFF70CBBFB
:1071C0000A9A131D16680A930123321E18BF012262
:1071D00036464FF00007FFF709BB0998594637AA12
:1071E000FFF7FEF800287FF4D7AA4C46FFF779BADC
:1071F0000998594637AAFFF7F3F800287FF4CCAA7C
:107200004C46FFF760BA302800F09682119A30237E
:1072100002F8013D169B11929B1A0E93FFF71BBBC0
:107220000998594637AAFFF7DBF800287FF4B4AA7B
:107230004C46FFF787BB5E60389A399901321F6070
:107240008919072A399138923FF7C1AB0833FFF704
:1072500071BA0A992B462A780A91FFF7B8B91AF041
:10726000100F00F0CD810A980D9900F1040A03680F
:107270001960FFF76DB90A9AD31D23F0070303F1D4
:1072800008000A905E681F68199610973FE41AF08C
:10729000400300F0A9810A9913460A1D0A920E883C
:1072A000321E18BF012236464FF00007FFF79EBA84
:1072B000119A636038992260399A01313891D31854
:1072C0000729399300F3628208340123429E6360E8
:1072D000389B399A01331B980132072B3893D8BF5A
:1072E00004F108032060399200F34682429A119912
:1072F00018988E191E60811A596039998A1A38991E
:10730000121839920131389107293FF760AB0833E1
:10731000FFF710BA5546DDF838A05C60389A399905
:1073200001321F600919072A3991389200F37F82D0
:1073300008331AF0010F3FF4FDA91B9901225A608E
:10734000389A19603999013238920131072A3991F6
:107350003FF73DAB0833FFF7EDB92D238DF80F3123
:10736000FFF7E8BB0998594637AAFFF739F8002814
:107370007FF412AA4B4656E5F4B100000123636086
:10738000389A4BF24423C0F200032360399B013248
:1073900038920133072A3993D8BF04F1080300F368
:1073A0007381429A2AB9189818B91AF0010F3FF45C
:1073B000C1A91B9901225A60389A19603999013282
:1073C00038920131072A399100F368810833429CD1
:1073D0006442002C40F38781102C9E4F40F3A08123
:1073E00010260DF1DC0803E0103C102C40F39881CE
:1073F0005E60389A399901321F601031072A39913D
:1074000003F108033892EFDD099859464246FEF72A
:10741000E7FF4B460028E7D0FFF7BEB9399B5E4631
:10742000002B3FF4BAA90998594637AAFEF7D8FFAE
:10743000FFF7B3B90A994AF0200A6A786B1C0A91DF
:10744000FFF7C5B838463146089302F0C3FE089BE3
:10745000002840F00181B8F1FF3F08BF08F107089C
:107460000ED0149A672A14BF00230123472A08BFAD
:1074700043F0010323B1B8F1000F08BF4FF001083A
:1074800033463A46CDE93A234AF4807A3B9B002BB7
:10749000C0F20A82002315931499662914BF0023B1
:1074A0000123462908BF43F001031293002B00F08B
:1074B0008A810323CDF82C800B990E970F960093A9
:1074C0000998DDE90E23019142A9029141A9039196
:1074D00040A9049100F0E8FA149AB2F1670318BFCA
:1074E0000123472A0CBF002303F0010311902BB99D
:1074F0001AF0010F08BFDDF800C11AD0119B0B98DC
:10750000129903EB000C29B11B78302B00F0D080CE
:10751000429B9C443846002200233146CDF820C0CF
:1075200003F050FCDDF820C0002800F07381CDF896
:1075300000C114981199672814BF0023012347281C
:1075400008BF43F00103C1EB0C011891002B00F0C0
:107550004A81429A12F1030F0E9202DB904580F2AB
:107560004B81149B023B14930E9A1498531E429322
:10757000002B8DF8F800C0F2D1812B228DF8F92074
:10758000092B00F362813FA930338DF8FB303023A3
:107590008DF8FA303EAB189ACB1A18991A935918ED
:1075A000012A0E9140F3CC810E9801300E9020EA12
:1075B000E0710B91159B002B00F0FD802D23002026
:1075C0008DF80F311590FFF750B90C9B5B420C936F
:1075D000FFF7CEBA0E9A00209DF80F3122EAE27230
:1075E00015900B92FFF740B90A98011D0A910668A1
:1075F000321E18BF012236464FF00007FFF7F6B8DB
:107600001AF0400F17BF0A9A0A990D9802F1040A5E
:1076100011BF136801F1040A0B680D9A14BF18809A
:107620001A60FEF795BF0998594637AAFEF7D8FEAB
:1076300000287FF4B1A84B460BE40998402101F0E3
:10764000FDFA30603061002800F08D8140237361C5
:10765000FEF767BFF4B1000003204BF224224BF287
:1076600020210B901498C0F20001C0F20002159383
:107670004728D8BF0A462AF0800A032111929DF8B4
:107680000F310E91FFF7F0B80998594637AAFEF767
:10769000A7FE00287FF480A84B4682E60998594649
:1076A00037AAFEF79DFE00287FF476A84B468EE6AB
:1076B0003846002200233146CDF820C003F082FB7B
:1076C000DDF820C000287FF423AF0B9AC2F101033C
:1076D00042931EE70998594637AAFEF781FE002813
:1076E0007FF45AA84B46189A11985A60389A3999DB
:1076F00018600132189838920918072A39913FF713
:1077000066A90833FFF716B80021159102F072FE42
:107710009DF80F3120EAE0720E900B92FFF7A4B8AB
:107720005C60389A1F60511C399A389112190729E8
:107730003992CFDC0833D6E716991198081A0E90C3
:10774000FFF789B8B8F1060F34BF414606214BF266
:107750003C22C0F2000221EAE1730E9111920B93D8
:10776000FFF763B90998594637AAFEF739FE002892
:107770007FF412A84B463BE40998594637AAFEF716
:107780002FFE00287FF408A84B46AFE5099859461C
:1077900037AAFEF725FE00287EF4FEAF4C4694E59E
:1077A000CDF8388028EAE8781590CDF82C809DF83F
:1077B0000F31FFF759B80E989DF80F3120EAE070AD
:1077C0000B90FFF751B8149A652A14BF00230123C8
:1077D000452A08BF43F00103002B32D008F1010312
:1077E0000B93022368E61498652862DD149A662AD2
:1077F0001CBF429B0E936FD0189A0E9B9A425BDC83
:107800001AF0010F40F0818023EAE37067210B90AA
:107810001491CFE6409B9C4598BF9C467FF689AE6D
:10782000302203F8012B9C454093FAD881E6099851
:10783000594637AAFEF7D4FD00287EF4ADAF4B467B
:1078400077E5CDF82C80023336E646F2676C0DF111
:10785000F700C6F2666C8CFB0321DA17C2EBA102BB
:1078600002EB8201A3EB410113463031092A00F8F3
:10787000011DF0DC3033421ED9B200F8011C079B19
:10788000934298BF0DF1FA017FF684AE02460DF1E6
:10789000FB0301E012F8011B03F8011C19460798CD
:1078A00001339042F6D875E62D2006F1004615907A
:1078B000F2E542990E9157E60E9918980029DABF21
:1078C0000E9AC2F1020301231B18672123EAE37217
:1078D0000E9314910B926DE6429800280E9038DDBD
:1078E000B8F1000F07D11AF0010F04BF20EAE071D0
:1078F0000B913FF45FAE0E9A66201490531C4344E4
:107900000E9323EAE3710B9154E60E9A67231493C6
:1079100001320E9222EAE2700B904BE62D225B427E
:107920008DF8F9202CE60A991A78D1F800800431F4
:107930000A91B8F1000FB8BF4FF0FF38FEF747BE0D
:107940001AF0010F04BF21EAE1730B933FF432AE4A
:107950002AE6B8F1000F0ED11AF0010F0BD1012267
:107960000B920E9226E609980C234FF0FF310D91F1
:107970000360FEF71ABF08F10203662023EAE371F1
:107980000E9314900B9115E62DE9F84F03690E69DB
:10799000824689469E4200F38380F21C01F1140561
:1079A00000F11404013E92008B18121803F1040830
:1079B000596850680131FEF707FB0746002839D0A7
:1079C00000239C461A46E958E0581FFA81FE4FEA08
:1079D000114B81B20EFB07CE51180BFB07FC0CEBD1
:1079E0001E4C1FFA8EFECEEB01011FFA8CF24FEAFD
:1079F0001C4CC2EB10421FFA81FE02EB21424EEA00
:107A00000241E1500433121459198845DBD2321D6A
:107A10000AEB8203596869B99C4209D25AF82220BC
:107A200012B105E01A681AB9043B013E9C42F9D331
:107A3000CAF810604946504601F086FD00282CDB4C
:107A4000002301379C46EA58E05891B2120C1FFA05
:107A500080F9C2EB1042C1EB0901614402EB214203
:107A600089B241EA0241E15004334FEA224C5A19EB
:107A70009045E8D2321D0AEB8203596869B99C42ED
:107A800009D25AF8222012B105E01A681AB9043B4B
:107A9000013E9C42F9D3CAF810603846BDE8F88F21
:107AA0000020BDE8F88F00BF2DE9F04F466AA1B075
:107AB0000446904699462D9D002E00F0238432689E
:107AC00082B1616A4FF0010C766820460B685660FF
:107AD0004A6819460CFA02F29A6001F06FFE636A76
:107AE00000221A60B9F1000638DB00232B6040F257
:107AF0000003C7F6F0731A4606EA0303934217D051
:107B00000022002340464946CDE9068903F05AF990
:107B1000002829D02C9801232E990360002900F019
:107B2000D080794B581E2E9A136021B0BDE8F08F9B
:107B30002C9842F20F730360B8F1000F00F09580AB
:107B40004BF25420C0F200002E990029EDD0C278EB
:107B5000C31C002AE7D000F10803E4E726F0004642
:107B60000123B1462B60C2E72046DDE906231EA9AA
:107B700000911FA9019101F073FEC6F30A558346D7
:107B8000002D7ED0DDE90601A5F57E751F9F073D1E
:107B900021F07F4323F4700343F07E51002341F42E
:107BA000E001199340F200030022C3F6F87302F0DB
:107BB000EDFC4FA3D3E9002302F09CFE4EA3D3E9D2
:107BC000002302F0E5FCCDE90801284602F02CFE76
:107BD0004BA3D3E9002302F08DFE02460B46DDE9FC
:107BE000080102F0D5FCCDE9080103F01DF90022DF
:107BF00000230646DDE9080103F0EEF840B1304607
:107C000002F012FEDDE9082303F0DCF800B9013EC2
:107C1000162E5BD901231893013FB7EB050A42BF2B
:107C2000CAF1000ACDF83CA04FF0000A01D40022AE
:107C30000F92002EC0F27183B24400231796159361
:107C40002A9B092B62D8052B40F377862A980027B8
:107C500004382A902A998B1E032B00F2DD83DFE87B
:107C600013F0A503D803D503C40326F07F4626F4FA
:107C70007006002E7FF464AF4BF24820C0F2000083
:107C800062E71F9F1E9BFB1803F586639D1C202D3A
:107C9000DCBFC5F1200008FA00F008DD1E3BC5F18D
:107CA000400216FA02F228FA03F342EA030002F055
:107CB000ABFDA5F586650122033D1992A1F1F8718E
:107CC00070E74BF24420C0F200002EE74BF2A823ED
:107CD000DDE90601C0F2000303EBC603D3E900238C
:107CE00003F07AF8002840F02083189094E700BF52
:107CF00061436F63A787D23FB3C8608B288AC63FB2
:107D0000FB799F501344D33F45B2000000234FF04E
:107D1000FF301F4601212A931190169108902B9352
:107D2000656A00236B602046696801F063FD636A41
:107D300028601B681093002F00F05B81002E40F339
:107D40002A844BF2A82306F00F02C0F2000335117B
:107D500003EBC20315F0100FD3E90001CDE90C01CC
:107D600000F0E7824BF28033DDE90601C0F2000348
:107D700005F00F054FF00308D3E9082302F0E4FEF5
:107D8000CDE91201BDB14BF28037DDE90C23C0F221
:107D9000000715F0010F1046194607D0D7E9002358
:107DA00008F1010802F0A6FD02460B4608376D10E7
:107DB000EFD1CDE90C23DDE90C23DDE9120102F05E
:107DC000C3FECDE90C011899002900F0DE8040F2D5
:107DD0000003DDE90C010022C3F6F0734FF000054B
:107DE00002F0FAFF08B14FF00105089A002AD4BF4B
:107DF000002505F00105002D00F0C780119B002B28
:107E000040F3F58040F200030022C4F22403DDE9D0
:107E10000C0102F06FFDCDE90C0108F10100711EAB
:107E2000129102F001FD02460B46DDE90C0102F061
:107E300061FD40F200030022C4F21C0302F0A8FB23
:107E4000DDF844C08046A1F15079169B002B00F06C
:107E5000AD834BF2A82340F20001C0F200030020E2
:107E600003EBCC03C3F6E071CDF80CC053E9022359
:107E700002F06AFE42464B46109D02F087FB8046A8
:107E80008946DDE90C0102F0CFFF074602F0CCFC89
:107E900002460B46DDE90C0102F078FB07F13003E6
:107EA000CDE90C01404605F8013B4946DDE90C23CC
:107EB00002F0B0FF002840F0138240F20001DDE93B
:107EC0000C230020C3F6F07102F060FB02460B4663
:107ED0004046494602F09EFFDDF80CC0002840F005
:107EE000E783BCF1010F40F38280CDF868B0012731
:107EF000CDF870A01D966646DDE90CAB0C9410E041
:107F000040F200010020C3F6F07102F03FFB424650
:107F10004B4602F061FF002840F0C783B74280F271
:107F20008B8440F20003404649460022C4F22403F9
:107F3000013502F0DFFC40F200030022C4F224030A
:107F4000804689465046594602F0D4FC8B4682460C
:107F500002F06AFF044602F067FC303402460B462A
:107F60005046594602F012FB109A4B46D4554246F1
:107F7000013782468B4602F02FFF52465B460028AF
:107F8000BED0DDF868B00C9CAAE1404602F04CFC83
:107F9000DDE90C2302F0AEFC40F200030022C4F243
:107FA0001C0302F0F5FA089AA1F150758046A94623
:107FB000002A40F0EC8240F20003DDE90C010022CF
:107FC000C4F2140302F0E2FA42462B46CDE90C015A
:107FD00002F020FF002840F04A824246DDE90C0111
:107FE00005F1004302F0F8FE002840F0D581DDE9FC
:107FF00006891E9B6FEA03074FEAD7770E2ECCBF88
:10800000002707F00107002F00F0B7802B984BF2F4
:10801000A823C0F20003089903EBC603C20F00298E
:10802000CCBF002202F00102D3E90001CDE9040136
:10803000002A40F0A08102460B464046494602F025
:1080400083FD109D02F0F0FE824602F0EDFBDDE9BB
:10805000042302F04FFC02460B464046494602F01C
:1080600095FA0AF1300305F8013B089A012A804687
:10807000894652D040F200030022C4F2240302F0E9
:1080800039FC00220023CDE9060102F09BFE002806
:1080900040F0EB8110984FF00108CDF82CB0A346CA
:1080A000871C0F96DDF82090DDE906450AE002F016
:1080B00021FC0022002304460D4602F083FE002826
:1080C00040F0CE81DDE904232046294608F101086D
:1080D00002F03AFD3E4602F0A7FE824602F0A4FB03
:1080E000DDE9042302F006FC02460B462046294641
:1080F00002F04CFA00220AF1300C07F801CC0137EB
:10810000C14540F20003C4F22403D0D135465C4699
:108110000F9E8046DDF82CB0894642464B464046CD
:10812000494602F035FA804689464246DDE90401B7
:108130004B4602F051FE60B9DDE9040142464B4670
:1081400002F040FE002800F090811AF0010F00F0CC
:108150008C81109900E01D4615F8012C6B1E392A00
:1081600040F067838B42F6D11099302301363122DB
:108170000B70109B1A701296B2E0169A002A40F00B
:10818000DF80159F0F9D0C92002DD4BF002301238B
:10819000BAF1000FD4BF002303F001034BB1AA458D
:1081A000B4BF53462B460F98C3EB0A0AED1AC01A08
:1081B0000F90159900291CDD169A002A00F0E9821B
:1081C000002F12DD0C993A46204601F073FD5A4605
:1081D0000C9020460C9901F085FC59460346204638
:1081E000039301F0EBFA039B9B46159BDA1B40F0CF
:1081F00011830121204601F00FFD069017980028F9
:1082000005DD06992046179A01F054FD06902A993B
:10821000012940F30A810027179B002B40F061825F
:108220000123534413F01F0340F02A811C230F9AAB
:108230009A44ED18D2180F920F9B002B05DD59467A
:108240001A46204601F0F0FB8346BAF1000F05DD27
:1082500006995246204601F0E7FB06901898002840
:1082600040F029822A9808990228D4BF00230123CC
:108270000029CCBF002303F00103002B00F00C8188
:10828000002940F08C8005220699089B204601F0C9
:10829000CDFC06905846069901F056F900287EDD7F
:1082A000109D01360027DDF830A0312305F8013B91
:1082B0000699204601F082FABAF1000F00F0D5804D
:1082C0003B1E18BF012357450CBF002303F00103D9
:1082D000002B40F0D0805146204601F06FFA1296F4
:1082E0002046594601F06AFA129A531C00222A705D
:1082F0002C982E990360002900F0D4812E9A1098B2
:10830000156012E4102000F091FCC66046608660A3
:10831000066006466062FFF7D2BB0F9871420022EA
:108320001591801B17920F908AE40021013E18914D
:1083300072E4DDE906234FF00208CDE9122321E5BE
:108340002A98012840F36C82089A1598531E984287
:10835000C0F25882C71A089B002BA8BF0F9DC0F21D
:1083600073820F9A204601219A44D2180F9201F08D
:1083700053FC0C9008E7089B73B940F200030022FD
:10838000C4F21403DDE9040102F0B4FA42464B469C
:1083900002F036FD00286AD0002206920C922B9B38
:1083A0000027DDF830A0DE43109D81E70021169103
:1083B0002B98002840F39F812B980146119008903C
:1083C000656A002217296A6040F2AB8204235B00D1
:1083D000013203F114008842F9D9089B6A600E2B20
:1083E0008CBF002707F001079DE4012216922B9B0A
:1083F000F3181193591C0029C8BF0891E0DC0E291D
:108400008CBF002707F00107089189E40123169328
:10841000CEE700221692EAE74FF0FF330027012053
:108420001193169008932B977AE4B8F1000F7FF41C
:10843000F2AE29F07F4323F47003002B7FF4EBAE00
:1084400040F20003C7F6F07309EA0303002B3FF480
:10845000E2AE0F9A0AF1010A012701320F92DBE620
:1084600035465C460F9EDDF82CB0129638E70020AA
:1084700006900C9014E73946204601F09FF92AE750
:10848000C3F12003042B40F354820F99043B9A4418
:10849000ED18C9180F91CFE61699002900F0318127
:1084A000002D05DD0C992A46204601F0BDFA0C90FE
:1084B000002F40F0EA81DDF830A0109D012308F084
:1084C00001000C9F11900F951D460C960699584679
:1084D000FFF75AFA394630300B90584601F034F81D
:1084E000069952460646204601F022FAC3688046A5
:1084F000002B3DD04FF001094146204601F05EF9C6
:108500002A9959EA010103D1119A002A00F0EB815E
:10851000002EC0F29E812A9A324303D1119B002B78
:1085200000F09781B9F1000F00F3CE810F990B9AFB
:1085300001F8012B089B0F919D4200F0C281594622
:108540000A220023204601F071FB57453946834635
:1085500014D00A2200232046013501F067FB514662
:108560000A2200230746204601F060FB8246ADE761
:108570005846414600F0E8FF8146BDE720460A2202
:108580000023013501F052FB074682469EE7129612
:10859000DDF820C059E47542002D40F00181DDE98D
:1085A00006014FF00208CDE90C010CE44BF2A821C2
:1085B0004246C0F200014B4601EBCC01CDF80CC0A5
:1085C000109D51E9020102F095F9CDE91A01DDE9AA
:1085D0000C0102F029FC074602F026F90B46024680
:1085E000DDE90C0101F0D2FF07F13003CDE90C0108
:1085F00005F8013BDDF80CC0BCF1010F29D0D146D4
:10860000DDE90C01B246109E1C9501276546A04687
:1086100040F200030022C4F2240302F06BF9CDE91A
:108620000C0102F001FC044602F0FEF83034024670
:108630000B46DDE90C0101F0A9FFF4550137AF420B
:10864000E6D11C9D013F56464446CA46ED19CDE988
:108650000C0140F200030022C3F6E073DDE91A01C9
:1086600001F096FF02460B46DDE90C0102F0D2FB59
:10867000F0B940F20001DDE91A230020C3F6E071F1
:1086800001F084FF02460B46DDE90C0102F0A4FB79
:1086900000283FF4ACAC2B461D4613F8012D302AC0
:1086A000FAD01DE61098FFF740BADDF868B00C9CD0
:1086B000129E109950E55846069900F045FF002893
:1086C000BFF6D0AD594620460A22002301F0AEFA8B
:1086D0001699013E8346002940F01981119A0892AB
:1086E000C0E50698036900EB8303186900F0DAFE21
:1086F000C0F1200395E50121119108912B91FFF71D
:108700000FBB109DB146169FAA46DDF81880089E43
:1087100002E001F08BFA834641465846FFF734F9F0
:1087200001350A220023594600F1300C0AF807C02F
:1087300001372046BE42ECDCDDF830A04E46002773
:10874000CDF82CC059460122204601F06DF906995A
:10875000834600F0F9FE00280FDD109900E01D4669
:1087600015F8012C6B1E392A40F08C808B42F6D113
:108770001099312301360B709AE503D10B9810F054
:10878000010FEAD12B461D4613F8012D302AFAD0ED
:108790008EE55946159A204601F08CFA834628E565
:1087A00005F00F034BF2A822C0F20002DDE906013A
:1087B00002EBC303D3E9002302F09CF82D1108BF9C
:1087C0004FF00208CDE90C013FF4FDAA4BF28037CF
:1087D000DDE90C234FF00208C0F2000715F0010F8D
:1087E0001046194607D0D7E9002308F1010802F026
:1087F00081F802460B4608376D10EFD1CDE90C2306
:10880000FFF7E1BA1599179A5B1AC918D218159192
:108810001792A0E55946204601F04CFA8346E8E459
:108820001999002947D003F58663159F03330F9DDF
:1088300097E50132D2B29DE4DDF868B0DDF870A0B2
:108840001D9E0C9CFFF7D3BB0F99002308980D1AAF
:1088500087E5B9F1000F0F9D0C9E0FDD59460122EF
:10886000204601F0E1F80699834600F06DFE0028ED
:1088700047DD0B99392931D001310B910B9A05F85D
:10888000012B15E501321A7012E50C9A2046516849
:1088900000F0B0FF0C9B03F10C011A690232920048
:1088A00005460C3000F0D6FC20462946012201F096
:1088B000BBF8824601E61F9B159F0F9DC3F136034F
:1088C0004FE50F9D0C9E3DE70B9B0F9D392B0C9E9A
:1088D00004D00B98431C05F8013BE9E4392305F863
:1088E000013B10993CE70B9833460F9D39280C9EAD
:1088F000F4D0002B01DD01300B900B9905F8011B22
:10890000D6E4BBD10B9810F0010FB7D0B1E700232C
:108910000C9920460A2201F089F9119B08930C90CA
:10892000A0E408990E298CBF002707F00107FFF784
:10893000FAB93FF481AC1C3379E40127FFF78AB917
:10894000F8B540F22414C1F200040F46054600F0C9
:10895000A5FDA3685E6826F0030606F57E630F3367
:10896000DF1B3F0B013F3F03B7F5805F07DB0021B3
:10897000284601F03DFCA368F318834204D0284642
:1089800000F08EFD0020F8BD7942284601F030FC51
:10899000B0F1FF3F10D0A26843F21403C1F200030C
:1089A000F61B46F00106284656601A68D71B1F6062
:1089B00000F076FD0120F8BD0021284601F018FCEA
:1089C000A368C21A0F2ADADD40F22C5443F21401D4
:1089D000C1F20004C1F2000142F001022468001B50
:1089E00008605A60CBE700BF2DE9F04105460C4610
:1089F000002900F0888000F051FDA4F1080240F247
:108A000024105668C1F2000026F00103D0F808C017
:108A1000D1188C454F6827F0030700F0958016F0B9
:108A200001064F605FD00026CC19646814F0010F76
:108A300006D1DB19002E7AD08C68C9688C60E160A1
:108A400043F00101D3505160002E47D1B3F5007FB0
:108A50005BD3590A04299EBF4FEA931C0CF1380CD2
:108A60004FEACC0428D914299CBF01F15B0C4FEAD2
:108A7000CC0421D954299EBF4FEA133C0CF16E0C53
:108A80004FEACC0418D9B1F5AA7F9EBF4FEAD33C78
:108A90000CF1770C4FEACC040ED940F2545C6145DE
:108AA00095BF4FEA934C4FF47C740CF17C0C4FF063
:108AB0007E0C98BF4FEACC040419A168A14203D1EF
:108AC00064E089688C4204D0486820F00300834247
:108AD000F7D3CB68D3609160CA609A602846BDE83E
:108AE000F04100F0DDBC54F8084C00F1080C121BFA
:108AF0001B199468644547D0D2F80CC0CCF80840E4
:108B0000C4F80CC090E7BDE8F081DB084FF0010C21
:108B1000466800EBC3019B100CFA03F3D1608C682C
:108B200046EA030343609460E2608A60D6E78C689B
:108B30001C4FBC4281D1D35043F00103E260A260DC
:108B400053609460D460C9E7FB1816F0010F07D199
:108B500054F8081C521A5B18D4689168A160CC6064
:108B600040F230518260C1F2000143F001005060D8
:108B70000A689342B2D343F210032846C1F20003BD
:108B80001968FFF7DDFEA9E701264DE701264468D5
:108B90004FEAAC0C0B4606FA0CFC44EA0C044460A9
:108BA00098E700BF2C0100104BF26023C0F20003D5
:108BB000186870470048704764B20000004870476A
:108BC00064B2000070B505460E46144672B14BF211
:108BD0005C211046C0F2000101F01EFB58B94BF2B7
:108BE0005C202C62C0F20000EE6170BD4BF25C2094
:108BF000C0F2000070BD4BF214212046C0F200010B
:108C000001F00AFB0028EAD0002070BD40F22003EA
:108C10000A46C1F2000301461868D3E740F2200378
:108C20000146C1F200031868FFF7DEBE40F22003E0
:108C30000146C1F20003186800F000B82DE9F04FBA
:108C400001F10B04162C83B006462FD80023102404
:108C50008C422CBF194643F00101002930D1304627
:108C600000F01CFCB4F5FC7F2ED24FEAD40E40F28B
:108C70002415C1F2000505EBCE02D368934200F043
:108C800006825A6803F10805D968304622F0030CC1
:108C90009A6863445C688A6044F00104D1605C6057
:108CA00000F0FEFB284603B0BDE8F08F24F0070477
:108CB000E30F8C422CBF194643F001010029CED0AE
:108CC0000C2300253360EDE75FEA542E04BF4FEA22
:108CD000D40E4FEACE0040F0908040F22415C1F24D
:108CE00000052818C368984206D10DE0002A80F2DA
:108CF0006F81DB68984207D0596821F003010A1B95
:108D00000F2AF3DD0EF1FF3E0EF1010E40F22417A3
:108D1000C1F2000707F108018B68994208BF7A6821
:108D200026D05A6822F0030CC4EB0C020F2A00F381
:108D30009481002AC960896080F29980BCF5007F27
:108D400080F065814FEADC0C4FF0010A7A6807EB8E
:108D5000CC004FEAAC0C0AFA0CFCD860D0F80880C2
:108D60004CEA02027A60C3F80880C8F80C308360CD
:108D70004FF0010C4FEAAE030CFA03FC944500F2ED
:108D8000828012EA0C0F08D12EF0030E4FEA4C0C31
:108D90000EF1040E12EA0C0FF8D007EBCE09F246E2
:108DA000C846D8F80C30984507D168E1002A80F20F
:108DB0007881DB68984500F06281586820F00300F4
:108DC000021B0F2AF2DD1D461F19D3F80CC044F018
:108DD000010E55F8084F3046BA5042F00102C3F870
:108DE00004E0CCF80840C4F80CC08F60CF607A6013
:108DF000B960F96000F054FB54E7BEF1040F9EBF68
:108E00004FEA941E0EF1380E4FEACE007FF665AFA2
:108E1000BEF1140F9CBF0EF15B0E4FEACE007FF641
:108E20005CAFBEF1540F9EBF4FEA143E0EF16E0EC2
:108E30004FEACE007FF651AFBEF5AA7F9EBF4FEA44
:108E4000D43E0EF1770E4FEACE007FF646AF40F2E9
:108E500054539E4595BF4FEA944E4FF47C700EF1EB
:108E60007C0E4FF07E0E98BF4FEACE0035E703EB45
:108E70000C0203F108053046536843F001035360C8
:108E800000F00EFB0EE7D7F80880D8F8043023F086
:108E90000309C4EB09024C4594BF002301230F2AA8
:108EA000D8BF43F00103002B00F0A18043F2100B68
:108EB000D5F80824C1F2000BDBF8003010331B1981
:108EC000B2F1FF3F06D003F57E631F3323F47E63C8
:108ED00023F01F0319463046019301F089F9019BE5
:108EE000B0F1FF3F824600F0F48008EB09018142B7
:108EF00000F2EC80DBF804209A185145CBF80420EE
:108F000000F04581D5F8085440F22410C1F2000069
:108F1000B5F1FF3F08BFC0F808A403D05244511A6E
:108F2000CBF804101AF00705304617BFC5F1080545
:108F30004FF48055AA4405F5805553441B051B0D7D
:108F4000ED1A294601F054F9B0F1FF3F00F02C81F1
:108F5000CAEB0001491941F00101DBF8042043F29A
:108F60001003C7F808A0C1F20003AA18B845CBF84F
:108F70000420CAF8041017D0B9F10F0F40F2DF80B7
:108F8000A9F10C01052521F0070108EB01000F29CB
:108F900085604560D8F8040000F0010041EA000057
:108FA000C8F8040000F2AC80D04643F21003DBF8AE
:108FB0002C10C1F200038A42DBF8301088BFDA625D
:108FC00043F21003C1F200038A4288BF1A6382E0B1
:108FD0005C189A68D9683046666803F108058A60AB
:108FE00046F00103D160636000F05AFA5AE608EBDC
:108FF000040342F0010244F001043046C8F8044082
:1090000008F108055A60BB6000F04AFA4AE64FEAE8
:109010005C22042A54D9142A00F289805B324FEA78
:10902000C208A84440F22417C1F20007D8F808008B
:10903000404503D16FE08068804504D0426822F04B
:1090400003029445F7D3D0F80CC0C3F80CC0986065
:109050007A68C360CCF808308AE61F19304644F0BD
:109060000104CF605C6003F10805BA5042F00102D0
:109070008F607A60B960F96000F012FA12E60AF1C6
:10908000010A1AF0030F5FD003F1080889E603F123
:109090000802D3689A4208BF0EF1020E3FF436AEC2
:1090A000EFE51D461918DA68304655F8083F4C6858
:1090B000936044F00104DA604C6000F0F1F9F1E5EE
:1090C0004FEA9C1238324FEAC208AAE7B8453FF48B
:1090D00011AFD7F80880D8F8042022F00302944298
:1090E00094BF00230123121B0F2AD8BF43F00103B2
:1090F000002B3FF47CAF3046002500F0D1F9D1E5DC
:1091000008F1080130460193FFF76EFC019BD7F888
:1091100008805A6849E74FF0010AD7F80480921096
:1091200084460AFA02F248EA02027A608DE7542A7B
:1091300024D84FEA1C326E324FEAC20871E701238D
:10914000D046CAF80430C6E74A461EF0030F13465D
:109150000EF1FF3E33D053F808299A42F5D07B68D0
:109160004FEA4C0C9C453FF68EAEBCF1000F3FF42D
:109170008AAE1CEA030F27D0D6460EE6B2F5AA7FC8
:1091800015D84FEADC3277324FEAC20849E70805C2
:10919000000D00287FF4B6AED7F808804B4443F0AA
:1091A0000103C8F8043000E701210025D5E640F2AC
:1091B000545082420DD94FF47C787E2231E77B688F
:1091C00023EA0C037B60CBE74FEA4C0C0AF1040A5C
:1091D000CFE74FEA9C427C324FEAC20821E700BF4A
:1091E00010F0030FC9B210B410D0002A2FD00378AA
:1091F0008B422AD0013A05E0002A28D00378013AB0
:109200008B4222D0013010F0030FF5D1032A11D97F
:1092100041EA012444EA0444036884EA0303A3F115
:10922000013C2CEA030313F0803F03D1043A0430DD
:10923000032AF1D85AB103788B4206D0013A32B1F1
:1092400010F8013F013A8B42F9D110BC7047002061
:10925000FBE700BF032A2DE9F0070BD83AB1002342
:1092600011F803C000F803C001339342F8D1BDE800
:10927000F007704782180C46034603E014F8011CFF
:1092800003F8011C03F003061946A4460133013418
:10929000002EF3D11CF00304634608BFC1EB020C9F
:1092A00068D06542C4F1040A0CEB050733464FEA67
:1092B000CA0A5CF805604FEAC408551A08E057F876
:1092C000044F264604FA0AF449EA0404CC50043355
:1092D0005C18032D26FA08F9A5F104050CEB03062A
:1092E000EDDC002302E0F15CE154013319199142F5
:1092F000F9D3BCE753F8404C41F8404C53F83C4C90
:1093000041F83C4C53F8384C41F8384C53F8344C45
:1093100041F8344C53F8304C41F8304C53F82C4C55
:1093200041F82C4C53F8284C41F8284C53F8244C65
:1093300041F8244C53F8204C41F8204C53F81C4C75
:1093400041F81C4C53F8184C41F8184C53F8144C85
:1093500041F8144C53F8104C41F8104C53F80C4C95
:1093600041F80C4C53F8084C41F8084C53F8044CA5
:1093700041F8044C1C460D4640334031BCF13F0FD0
:10938000ACF1400CB6DC21462B46541B0FE051F8E3
:10939000105C43F8105C51F80C5C43F80C5C51F81D
:1093A000085C43F8085C51F8045C43F8045C0F2C3B
:1093B0000D469C4601F1100103F11003A4F11004C5
:1093C000E5DCCCEB0201002303E0EC584CF8034051
:1093D00004335E19032903EB0C04A1F10401F4DC4E
:1093E0007FE700BF88428C4670B4054614460ED90C
:1093F0008B1898420BD242B1C2EB030C0146531EAC
:109400001CF80320CA54013BFAD270BC70470F2AE3
:1094100009D8002CF9D000231CF80320EA540133AA
:10942000A342F9D1F1E741EA000313F0030FF0D1B1
:1094300094460C4603462568ACF1100C1D60656827
:109440005D60A5689D60E5681034DD601033BCF197
:109450000F0FF0D8103A4FEA121C0CF10105CCEBBB
:109460000C7C2D0102EB0C1601EB050C4519032EAB
:109470003446CED900235CF80320EA500433F21AB4
:10948000032AF8D8043EB3085A1CC3EB8373920036
:10949000944406EB8304AD18BBE700BF704700BFE0
:1094A000704700BF020C03461204B2B1002013F053
:1094B0007F4F01D108301B0213F0704F01D10430EF
:1094C0001B0113F0404F01D102309B00002B03DB46
:1094D00013F0804F04D00130704703041020E6E7FA
:1094E000202070470368024613F0070009D013F0EC
:1094F000010F21D113F0020F22D19B08022013602B
:10950000704799B209B91B0C102013F0FF0F01D15D
:1095100008301B0A13F00F0F01D104301B0913F0A0
:10952000030F01D102309B0813F0010F02D15B0839
:1095300004D001301360704700207047202070472E
:109540005B0801201360704703460A69006910B484
:10955000801A11D1043203F1140C92009B1889185F
:109560000431043353F8044C043B51F8042C0439FF
:10957000944203D19C45F5D310BC704738BF4FF0DF
:10958000FF30F9D30120F7E740F20003C7F6F0738C
:1095900001EA0303A3F15073002B02DD19460020FA
:1095A00070475B421B15132B0EDD143B1E2B03DD96
:1095B00001230021184670470122C3F11F03002137
:1095C00012FA03F3184670474FF40022002052FAB3
:1095D00003F170472DE9F041046900F114060F46CC
:1095E000043450F8245000EB8404A0462846FFF7CA
:1095F00059FF0A28C0F120033B6014DCA642C0F1E9
:109600000B0337D254F8041CD94025FA03FC15305B
:109610004CF07E53854043F4E00341EA05021046D6
:109620001946BDE8F081A64220D300210B3802BFC5
:1096300045F07E530A4643F4E003F0D0B442C0F153
:10964000200319D954F8044CDC40854021FA03FC6E
:1096500045F07E5511FA00F045F4E00544EA0002B9
:1096600045EA0C0310461946BDE8F08154F8041C85
:10967000043CDBE70021C8E70024E6E72DE9F043DE
:1096800083B00E4601A90746FFF7A4FF0D46044626
:1096900069463046FFF79EFFDDF804C0A946A046A4
:1096A0000B4602463169164638691F46401A009932
:1096B000C1EB0C0101EB40110029C9BF05EB0159B9
:1096C000A3EB015724464D46DCBF12463B462046DD
:1096D000294601F039FA03B0BDE8F083172810B528
:1096E00004460EDD40F200010020C3F6F07140F2A6
:1096F00000030022C4F2240301F0FCF8013CF6D17F
:1097000010BD4BF2A823C0F2000303EBC003D3E962
:10971000000110BD1369013902F1140C10B402EB01
:1097200083024C1114320134944500EB84040FD2AF
:1097300000235CF80310C150043303EB0C018A4290
:10974000F7D86FEA0C0C624422F00302043280184E
:10975000844204D9002340F8043B8442FBD810BC67
:10976000704700BF02694B119A4210DB0EDD11F009
:109770001F010BD01A4600EB83035B6923FA01FC3F
:109780000CFA01F1994202D0012070471A460432C6
:1097900000F1140100EB820303F1040C61450BD2CC
:1097A00050F82220002AEFD1994205D253F8042D17
:1097B000002AE9D19942F9D30020704730B5456AB3
:1097C00083B0044655B139B1636A4A68DB6853F81F
:1097D0002200086043F8221003B030BD1020019130
:1097E000FFF724FA01996062C560456085600560F5
:1097F000E9E700BF70B5446A06460D4664B1E26809
:10980000A2B152F82530EBB1196842F825100022B8
:10981000DA601A61184670BD1020FFF707FA0023BE
:1098200004467062C3604360836003601022304668
:10983000042100F00FFE736AE060DA68002AE0D1CC
:109840001346E7E7012430462146AC40621D9200F2
:1098500000F000FE03460028DCD045608460D6E7B7
:109860002DE9F04583B001211D4614460A9F0B9E49
:10987000FFF7C0FF25F0004225F07F4323F470037B
:1098800015465FEA125A00931CBF43F480130093FD
:109890008046002C23D002A840F8044DFFF722FE9A
:1098A0000346002837D10199009AC8F81410002AFD
:1098B00014BF02240124C8F81820C8F81040BAF1D7
:1098C000000F1BD0AAF5866AC3F13502AAF1030A7C
:1098D00053443B603260404603B0BDE8F0856846C3
:1098E000FFF700FE01231C46C8F81030009BC8F8A3
:1098F000143000F12003BAF1000FE3D108EB840229
:10990000A3F58663023B3B601069FFF7CBFDC0EB1C
:1099100044103060DFE7009AC0F1200112FA01F133
:10992000C24001980143C8F814100092BFE700BF7D
:109930002DE9F84F13690F690C461546FF1A002FE1
:109940004FD06ADB002701F114066168FFF752FF70
:10995000D5F81080D4F810C005F11401002205EBF1
:10996000880504EB8C0405F11408143400F1140389
:10997000C76051F8047B56F8045BBB461FFA87FAB0
:109980003F0C1FFA85F9C7EB1547CAEB090A524489
:1099900007EB224792B242EA074243F8042B3A14FB
:1099A0008845E6D8A6420ED256F8041B8DB2090CA3
:1099B000521901EB224192B242EA014243F8042BD0
:1099C0000A14B442F0D853F8042C32B953F8082CD6
:1099D0000CF1FF3C043B002AF8D0C0F810C0BDE8F1
:1099E000F88F043301F114069B00D218CB1804330E
:1099F000043253F804CC043B52F8041C043A8C455E
:109A00000AD19E42F5D30021FFF7F4FE0123036142
:109A100000234361BDE8F88F97D223462C460127E7
:109A20001D4604F1140690E72DE9F8450D698B6891
:109A3000561101350C46AD1990469D428246496843
:109A400003DD5B0001319D42FBDC5046FFF7D2FE97
:109A5000002E074600F114020ADD0023194642F8E1
:109A600023100133B342FAD107EB830303F114024D
:109A7000206904F1140304EB8000143018F01F086F
:109A80001BD0C8F1200E00211E6806FA08FC41EA2E
:109A90000C0142F8041B53F8041B984221FA0EF102
:109AA000F2D8116001B101355046013D21463D61BA
:109AB000FFF784FE3846BDE8F88553F8081042F8F1
:109AC000081008F1040808EB03018842ECD953F8A8
:109AD000081042F8081008F1040808EB0301884256
:109AE000EBD8E1E72DE9F04FD1F8108017690D466A
:109AF000164687B0B845B5BF15463B460B464746A8
:109B0000B4BF1E469846AB6808EB070469689C42E0
:109B1000C8BF0131FFF76EFE00EB840300F1140BA8
:109B2000143303909B45049306D204995B460022AC
:109B300043F8042B9942FBD806EB880806F1140978
:109B400008F1140805EB870C1435C145CDF80480E5
:109B50000CF1140C02954BD24FF0000A059459F801
:109B60000A400AEB0B08A0B2D8B1029A434600247F
:109B700052F8045B1968AFB22D0C8EB2090C00FBD1
:109B8000076600FB0511361901EB1641B6B20C0C45
:109B9000944546EA014643F8046BE9D81C6059F83D
:109BA0000A40240C1CD05BF80A204146029B002589
:109BB00010461E8897B206FB045505EB104547EA90
:109BC00005470F6051F8040F53F8042B86B2120CAE
:109BD00002FB046202EB1542150C9C45E9D80A60B1
:109BE0000AF1040A019A0AEB09039A42B7D8059CC4
:109BF000002C0BDD049A52F8043C3BB9134603E0F9
:109C000053F8082C043B0AB9013CF9D1039B1846D0
:109C10001C6107B0BDE8F08F10B50C460121FFF7BD
:109C2000E9FD01224461026110BD00BF2DE9F0454C
:109C30000D46002106462C6983B005F1140808463C
:109C400058F8017001301FFA87FA4FEA174C0AFBE7
:109C500002330CFB02FC0CEB134C9BB203EB0C43EA
:109C600048F80130043184424FEA1C43E8DC3BB140
:109C7000AA68944208DA05EB840201342C6153612E
:109C8000284603B0BDE8F08569683046019301318C
:109C9000FFF7B0FD2A6905F10C0102329200074678
:109CA0000C30FFF7D7FA294630463D46FFF786FDD0
:109CB000019BE0E72DE9F041154612F0030204464E
:109CC00088462CD1AD101ED0666A002E34D0B768FD
:109CD000002F3BD015F0010F08D16D1013D03E6856
:109CE000A6B13046074615F0010FF6D041463A4678
:109CF0002046FFF7F7FE414606462046FFF75EFD89
:109D00006D10B046EBD14046BDE8F08139463A4689
:109D10002046FFF7E7FE386007460660E3E74BF2B0
:109D2000A82C0023C0F2000C0CEB8202D2F8C42055
:109D3000FFF77CFF8046C5E71020FEF777FF002382
:109D400006466062C360436083600360204640F261
:109D50007121FFF761FF0023B06007460360B9E798
:109D60002DE9F8451E4648F6396306F1080CC3F69E
:109D7000E30388460546174683FB0C134FEAEC7C49
:109D8000CCEB630CBCF1010F35DD00210122520048
:109D900001319445FBDC2846FFF72CFD089B43610D
:109DA0000123092F036122DD08F1090A092418F8AB
:109DB000043001460A220134303B2846FFF736FFC3
:109DC000A742F4DC0AEB0708A8F10808BE420CDD44
:109DD000002418F80430014601340A22303B28469A
:109DE000FFF724FFE3199E42F3DCBDE8F88508F194
:109DF0000A080927EAE70021CDE700BF2DE9F04F67
:109E0000914683B007460E46002900F03A81A1F141
:109E1000080809F10B04FFF741FB162CD8F80410D1
:109E20000B4600F2A0801022002514464C4538BF96
:109E300045F00105002D40F02A8121F0030A9245EA
:109E4000A2BF4046554608F1080875DA40F22413CF
:109E500008EB0A00C1F20003D3F808E0864500F0E1
:109E60001A81D0F804C02CF0010B8344DBF804B055
:109E70001BF0010F7CD0AC46284611F0010F40F0DA
:109E80009B8056F8081CC1EB080BDBF8045025F04A
:109E90000305002800F0DD80704500F01F8105EB10
:109EA0000A030CEB03059542B8BF1D46C0F2D280F1
:109EB00081685B46C068AAF10402242A8160C860F8
:109EC00053F8081FDBF80C008160C86000F2D080F6
:109ED000132A9C4621D931460BF1100C51F8040B82
:109EE000CBF8080070680E1D1B2ACBF80C0014D9A3
:109EF0004868311D0BF1180CCBF8100070680E1D6E
:109F0000242ACBF8140008D14A680BF1200CCBF8B6
:109F1000182072680836CBF81C20314698466246F5
:109F2000584651F8043B42F8043B7368CCF80430BF
:109F30004B685360DBF80430C4EB050CBCF10F0F29
:109F400026D8421903F0010343EA0505456053682A
:109F500043F00103536038464546FFF7A1FA28460F
:109F600003B0BDE8F08F24F007042246E50F5DE75B
:109F70002CF0030C0CEB0A059542FFF67EAF8268CD
:109F80000B46C168404608F108088A60D160D3E7F3
:109F9000011903F0010301EB0C0243EA04044CF045
:109FA000010344604B6038465368083143F00103B5
:109FB0005360FEF719FDCEE749463846FEF73EFEF0
:109FC0000546002841D0D8F80430A0F1080223F05B
:109FD000010141448A4200F0D780AAF104023146CF
:109FE000242A78D8132A034621D9344654F8043B4E
:109FF000211D40F8043B031DD6F804C01B2AC5F8F8
:10A0000004C014D9D4F804E01C1D01F1040CC0F8FC
:10A0100004E048680CF104015860231D242A06D18D
:10A02000DCF8042062604A6808315A600833084648
:10A030001A4650F8044B42F8044B4968596043688B
:10A04000536031463846FEF7CFFC3846FFF728FA12
:10A0500085E755449542AFDB5B46DBF80C00AAF17F
:10A06000040253F8081F242A8160C8607FF630AFCD
:10A07000184631469846FFF7B5F95846DBF80430E4
:10A080005AE7114603B0BDE8F04FFEF7D7BD0C23E9
:10A0900000253B6063E7DEF8045004F1100B25F067
:10A0A000030C0CEB0A005845B8BF7046FFF6E5AE4E
:10A0B00008EB0402011B41F001019A60516038462F
:10A0C000D8F80410354601F001031C43C8F80440D9
:10A0D000FFF7E6F943E7FFF785F9B2E7554404F1E6
:10A0E0001001AC448C45B5DB5D46DBF80C00AAF1F1
:10A0F000040255F8081F242A8160C8604CD8132A2E
:10A10000284624D931460BF1100051F804EBCBF866
:10A1100008E0D6F804E00E1D1B2ACBF80CE016D997
:10A12000D1F804E0311D0BF11800CBF810E0D6F89F
:10A1300004E00E1D242ACBF814E008D14A680BF184
:10A140002000CBF8182072680836CBF81C20314666
:10A15000024651F804EB42F804EB76684660496821
:10A1600051600BEB0402C4EB0C0141F001019A6059
:10A1700051603846DBF8041001F001031C43CBF8B2
:10A180000440FFF78DF9EAE65568404608F10808F3
:10A1900025F003055544CFE6314628460093CDF817
:10A1A00004C0FFF71FF9DDF804C0009BD9E700BF2A
:10A1B0000246404240EA020321F0004141EAD373E3
:10A1C000C3F1FE4303F57003584240EA0303D81776
:10A1D0000130704702464042104321F0004141EAFD
:10A1E000D070C0F1FE4000F57000C00F704700BF96
:10A1F00038B543F2B414C1F2000405460846002302
:10A200002360F7F73BFBB0F1FF3F00D038BD236878
:10A21000002BFBD02B6038BD80EA010212F0030F47
:10A220003AD110F0030220F0030021F0030150F8AE
:10A2300004CB08BF51F8043B0DD082F003024FEA73
:10A24000C2026FF07F4323FA02F251F8043B4CEA5A
:10A25000020C43EA020300BFACF101329C4501BF8E
:10A2600022EA0C0212F0803F50F804CB51F8043B74
:10A27000F2D04FEA0C604FEA1C2C012828BFB0EB4B
:10A28000036F08BF1B0AF4D003F0FF034FEA10600E
:10A29000A0EB0300704700BF10F0030F0AD010F8C6
:10A2A000012B11F8013B012A28BF9A42F4D0A2EBFE
:10A2B000030070474DF8045D4DF8044D4FF0010266
:10A2C00042EA022242EA024201F0030C21F00301B9
:10A2D00050F8044B51F8045BBCF1020F26D04BD868
:10A2E00024F07F4CBCEB152FA4EB020323EA0403FC
:10A2F0000DD113EAC21308BF51F8045B0AD18CEAEE
:10A30000040CBCEB056F0CD150F8044BE8E74FEAA6
:10A3100015255CE033F07F4352D10D784FEA146C81
:10A3200055E04FEA146C05F0FF0550E04FEA044C8D
:10A33000A4EB02034FEA1C4C23EA0403BCEB154FC9
:10A3400017D113EAC21308BF51F8045B07D18CEA96
:10A35000040CBCEB054F08D150F8044BE6E71B0496
:10A360002ED10D884FEA144C31E04FEA05454FEAF3
:10A37000144C4FEA15452AE004F0FF0CBCEB156FB6
:10A38000A4EB020323EA04030DD113EAC21308BFAE
:10A3900051F8045B0AD18CEA040CBCEB052F0AD1FE
:10A3A00050F8044BE8E74FEA156510E014F0FF0F92
:10A3B00006D051F8045B4FEA142C25F07F4506E0E7
:10A3C0004FF000005DF8044B5DF8045B70470CF043
:10A3D000FF0205F0FF00012828BF904204BF4FEAAA
:10A3E0001C2C2D0AF3D0A2EB00005DF8044B5DF8A5
:10A3F000045B704720F0030110F00300C0F100007F
:10A4000051F8043B00F1040C4FEACC0C6FF0000251
:10A410001CBF22FA0CF213434FF0010C4CEA0C2C37
:10A420004CEA0C4CA3EB0C0222EA030212EACC1217
:10A4300004BF51F8043B0430F4D013F0FF0F1FBFEA
:10A44000013013F47F4F013013F47F0F18BF013038
:10A45000704700BF38B501FB02F1FEF7EFFB044681
:10A46000F8B150F8042C22F00302043A242A1AD836
:10A47000132A03460FD9002140F8041B031D1B2A91
:10A48000616008D91D1D416059602B1D242A02BF3F
:10A490006960596008331A46002142F8041B59606C
:10A4A0005160204638BD002100F002F8204638BD3A
:10A4B000032AC9B230B407D822B10023C1540133F2
:10A4C0009342FBD130BC704700EB020C034601E025
:10A4D00003F8011C03F003041A460133002CF7D1E2
:10A4E0004FF00133C2EB0C0403FB01F31FE042F811
:10A4F000403C42F83C3C42F8383C42F8343C42F89C
:10A50000303C42F82C3C42F8283C42F8243C42F8CB
:10A51000203C42F81C3C42F8183C42F8143C42F8FB
:10A52000103C42F80C3C42F8083C42F8043C15460A
:10A5300040323F2CA4F14004D9DC2A46C5EB0C0480
:10A5400007E042F8103C42F80C3C42F8083C42F864
:10A55000043C154610320F2CA4F11004F1DC2A46FD
:10A56000C5EB0C0501E042F8043C14460432032D0F
:10A57000A5F10405F7DC01E004F8011B6445FBD3F9
:10A58000A0E700BF81F0004102E000BF83F000437C
:10A5900030B54FEA41044FEA430594EA050F08BF7E
:10A5A00090EA020F1FBF54EA000C55EA020C7FEA42
:10A5B000645C7FEA655C00F0E2804FEA5454D4EBBF
:10A5C0005555B8BF6D420CDD2C4480EA020281EA89
:10A5D000030382EA000083EA010180EA020281EAC1
:10A5E0000303362D88BF30BD11F0004F4FEA013113
:10A5F0004FF4801C4CEA113102D0404261EB410122
:10A6000013F0004F4FEA03334CEA133302D05242A7
:10A6100063EB430394EA050F00F0A780A4F1010463
:10A62000D5F1200E0DDB02FA0EFC22FA05F280189D
:10A6300041F1000103FA0EF2801843FA05F3594183
:10A640000EE0A5F120050EF1200E012A03FA0EFC02
:10A6500028BF4CF0020C43FA05F3C01851EBE3712C
:10A6600001F0004507D54FF0000EDCF1000C7EEB49
:10A6700000006EEB0101B1F5801F1BD3B1F5001F87
:10A680000CD349085FEA30004FEA3C0C04F10104A6
:10A690004FEA445212F5800F80F09A80BCF1004FCF
:10A6A00008BF5FEA500C50F1000041EB045141EA51
:10A6B000050130BD5FEA4C0C404141EB010111F452
:10A6C000801FA4F10104E9D191F0000F04BF0146FD
:10A6D0000020B1FA81F308BF2033A3F10B03B3F1DB
:10A6E00020020CDA0C3208DD02F1140CC2F10C026B
:10A6F00001FA0CF021FA02F10CE002F11402D8BFC9
:10A70000C2F1200C01FA02F120FA0CFCDCBF41EA94
:10A710000C019040E41AA2BF01EB0451294330BD63
:10A720006FEA04041F3C1CDA0C340EDC04F1140440
:10A73000C4F1200220FA04F001FA02F340EA030017
:10A7400021FA04F345EA030130BDC4F10C04C4F15D
:10A75000200220FA02F001FA04F340EA030029463D
:10A7600030BD21FA04F0294630BD94F0000F83F487
:10A77000801306BF81F480110134013D4EE77FEA6A
:10A78000645C18BF7FEA655C29D094EA050F08BFB6
:10A7900090EA020F05D054EA000C04BF1946104697
:10A7A00030BD91EA030F1EBF0021002030BD5FEADB
:10A7B000545C05D14000494128BF41F0004130BD03
:10A7C00014F580043CBF01F5801130BD01F0004557
:10A7D00045F0FE4141F470014FF0000030BD7FEACA
:10A7E000645C1ABF194610467FEA655C1CBF0B46C5
:10A7F000024650EA013406BF52EA033591EA030FDC
:10A8000041F4002130BD00BF90F0000F04BF0021D3
:10A81000704730B54FF4806404F132044FF0000506
:10A820004FF0000150E700BF90F0000F04BF00217F
:10A83000704730B54FF4806404F1320410F00045E5
:10A8400048BF40424FF000013EE700BF42004FEAE0
:10A85000E2014FEA31014FEA02701FBF12F07F435D
:10A8600093F07F4F81F06051704792F0000F14BF5A
:10A8700093F07F4F704730B54FF4607401F000459E
:10A8800021F0004120E700BF50EA010208BF7047F5
:10A8900030B54FF000050AE050EA010208BF7047EA
:10A8A00030B511F0004502D5404261EB41014FF453
:10A8B000806404F132045FEA915C3FF4DCAE4FF057
:10A8C00003025FEADC0C18BF03325FEADC0C18BF3E
:10A8D000033202EBDC02C2F1200300FA03FC20FA8F
:10A8E00002F001FA03FE40EA0E0021FA02F11444DC
:10A8F000C1E600BF70B54FF0FF0C4CF4E06C1CEAF1
:10A9000011541DBF1CEA135594EA0C0F95EA0C0F65
:10A9100000F0DEF82C4481EA030621EA4C5123EAD8
:10A920004C5350EA013518BF52EA033541F4801107
:10A9300043F4801338D0A0FB02CE4FF00005E1FBBA
:10A9400002E506F00042E0FB03E54FF00006E1FB04
:10A9500003569CF0000F18BF4EF0010EA4F1FF0447
:10A96000B6F5007F64F5407404D25FEA4E0E6D4187
:10A9700046EB060642EAC62141EA55514FEAC52098
:10A9800040EA5E504FEACE2EB4F1FD0C88BFBCF514
:10A99000E06F1ED8BEF1004F08BF5FEA500E50F1C5
:10A9A000000041EB045170BD06F0004646EA01018B
:10A9B00040EA020081EA0301B4EB5C04C2BFD4EBBD
:10A9C0000C0541EA045170BD41F480114FF0000EB6
:10A9D000013C00F3AB8014F1360FDEBF002001F024
:10A9E000004170BDC4F10004203C35DA0C341BDC9E
:10A9F00004F11404C4F1200500FA05F320FA04F070
:10AA000001FA05F240EA020001F0004221F00041A3
:10AA100010EBD37021FA04F642EB06015EEA430E16
:10AA200008BF20EAD37070BDC4F10C04C4F1200546
:10AA300000FA04F320FA05F001FA04F240EA0200F9
:10AA400001F0004110EBD37041F100015EEA430ECA
:10AA500008BF20EAD37070BDC4F1200500FA05F2EA
:10AA60004EEA020E20FA04F301FA05F243EA020369
:10AA700021FA04F001F0004121FA04F220EA020078
:10AA800000EBD3705EEA430E08BF20EAD37070BDBE
:10AA900094F0000F0FD101F00046400041EB01019E
:10AAA00011F4801F08BF013CF7D041EA060195F080
:10AAB000000F18BF704703F00046520043EB03033A
:10AAC00013F4801F08BF013DF7D043EA0603704727
:10AAD00094EA0C0F0CEA135518BF95EA0C0F0CD032
:10AAE00050EA410618BF52EA4306D1D181EA030178
:10AAF00001F000414FF0000070BD50EA410606BF72
:10AB00001046194652EA430619D094EA0C0F02D1B6
:10AB100050EA013613D195EA0C0F05D152EA0336FB
:10AB20001CBF104619460AD181EA030101F0004119
:10AB300041F0FE4141F470014FF0000070BD41F062
:10AB4000FE4141F4780170BD70B54FF0FF0C4CF43C
:10AB5000E06C1CEA11541DBF1CEA135594EA0C0F5B
:10AB600095EA0C0F00F0A7F8A4EB050481EA030EA8
:10AB700052EA03354FEA013100F088804FEA03338F
:10AB80004FF0805545EA131343EA12634FEA02225D
:10AB900045EA111545EA10654FEA00260EF000411E
:10ABA0009D4208BF964244F1FD0404F5407402D270
:10ABB0005B084FEA3202B61A65EB03055B084FEA01
:10ABC00032024FF480104FF4002CB6EB020E75EBFE
:10ABD000030E22BFB61A754640EA0C005B084FEA26
:10ABE0003202B6EB020E75EB030E22BFB61A7546A3
:10ABF00040EA5C005B084FEA3202B6EB020E75EBEE
:10AC0000030E22BFB61A754640EA9C005B084FEA65
:10AC10003202B6EB020E75EB030E22BFB61A754672
:10AC200040EADC0055EA060E18D04FEA051545EA61
:10AC300016754FEA06164FEAC30343EA52734FEA0A
:10AC4000C2025FEA1C1CC0D111F4801F0BD141EA83
:10AC500000014FF000004FF0004CB6E711F4801FE8
:10AC600004BF01430020B4F1FD0C88BFBCF5E06FC8
:10AC70003FF6AFAEB5EB030C04BFB6EB020C5FEAD8
:10AC8000500C50F1000041EB045170BD0EF0004E2D
:10AC90004EEA113114EB5C04C2BFD4EB0C0541EA5F
:10ACA000045170BD41F480114FF0000E013C90E65C
:10ACB00045EA060E8DE60CEA135594EA0C0F08BF20
:10ACC00095EA0C0F3FF43BAF94EA0C0F0AD150EA1F
:10ACD00001347FF434AF95EA0C0F7FF425AF1046B2
:10ACE00019462CE795EA0C0F06D152EA03353FF4DA
:10ACF000FDAE1046194622E750EA410618BF52EA57
:10AD000043067FF4C5AE50EA41047FF40DAF52EA2A
:10AD100043057FF4EBAE12E74FF0FF3C06E000BFC7
:10AD20004FF0010C02E000BF4FF0010C4DF804CDD4
:10AD30004FEA410C7FEA6C5C4FEA430C18BF7FEA94
:10AD40006C5C1BD001B050EA410C0CBF52EA430CC2
:10AD500091EA030F02BF90EA020F0020704710F142
:10AD6000000F91EA030F58BF994208BF90422CBFD1
:10AD7000D8176FEAE37040F0010070474FEA410CCA
:10AD80007FEA6C5C02D150EA013C07D14FEA430CE8
:10AD90007FEA6C5CD6D152EA033CD3D05DF8040B59
:10ADA000704700BF8446104662468C46194663468B
:10ADB00000E000BF01B5FFF7B7FF002848BF10F162
:10ADC000000F01BD4DF808EDFFF7F4FF0CBF0120A7
:10ADD00000205DF808FB00BF4DF808EDFFF7EAFF23
:10ADE00034BF012000205DF808FB00BF4DF808EDDE
:10ADF000FFF7E0FF94BF012000205DF808FB00BFD3
:10AE00004DF808EDFFF7CEFF94BF012000205DF85C
:10AE100008FB00BF4DF808EDFFF7C4FF34BF012069
:10AE200000205DF808FB00BF4FEA410212F5001256
:10AE300015D211D56FF47873B3EB625212D94FEA81
:10AE4000C12343F0004343EA505311F0004F23FA6B
:10AE500002F018BF404270474FF00000704750EAC0
:10AE6000013005D111F0004008BF6FF0004070477D
:10AE70004FF00000704700BF08B500F04BF80748DE
:10AE800000B10068064901B109680022F5F790FE9B
:10AE9000044B0BB1AFF30080FEE700BF00000000E1
:10AEA000000000000000000080B51448144B21E0B1
:10AEB0005C689968DD688C420CD0002205E0A61819
:10AEC0000832D6E9008941E902898C460831AA4254
:10AED000F5D101E004EB050C1C696146002204E099
:10AEE00008320026002741E902670831A242F7D163
:10AEF000143301380028DBD1FFF7BEFF010000004A
:10AF0000F0B3000001498D46014908470080001058
:10AF1000A9AE000070B54BF2DC364BF2DC35C0F266
:10AF20000006C0F20005761BB61006D0002455F8C6
:10AF3000243001349847A642F9D84BF2DC354BF265
:10AF4000E036C0F20005C0F20006761B00F040FAC1
:10AF5000B61006D0002455F8243001349847A64294
:10AF6000F9D870BD5278206F76657272756E0000E8
:10AF70005278206572726F723A2000005278206613
:10AF8000696E697368000000527820646F6E650016
:10AF9000547820756E6465722D72756E0000000025
:10AFA0005478206572726F72000000005478206639
:10AFB000696E697368000000547820646F6E6500E4
:10AFC000496E697420454D4143206D6F64756C6511
:10AFD000000000004D41435B312E2E365D20616440
:10AFE00064723A2025582D25582D25582D25582D89
:10AFF00025582D2558200A0D000000004572726F5B
:10B000007220647572696E6720696E697469616C1B
:10B01000697A696E6720454D41432C2072657374CF
:10B020006172742061667465722061207768696C52
:10B0300065000000496E697469616C697A65204534
:10B040004D414320636F6D706C65746500000000B6
:10B05000456E74657220536C656570206D6F646514
:10B06000206E6F772E2E2E0057616B652075702035
:10B0700066726F6D20736C656570206D6F6465001E
:10B0800053656E64207061636B6574000102030494
:10B09000050600005278206F76657272756E0000AA
:10B0A0005278206572726F723A20000052782066E2
:10B0B000696E697368000000527820646F6E6500E5
:10B0C000547820756E6465722D72756E00000000F4
:10B0D0005478206572726F72000000005478206608
:10B0E000696E697368000000547820646F6E6500B3
:10B0F000496E697420454D4143206D6F64756C65E0
:10B10000000000004D41435B312E2E365D2061640E
:10B1100064723A2025582D25582D25582D25582D57
:10B1200025582D2558200A0D000000004572726F29
:10B130007220647572696E6720696E697469616CEA
:10B14000697A696E6720454D41432C20726573749E
:10B150006172742061667465722061207768696C21
:10B1600065000000496E697469616C697A65204503
:10B170004D414320636F6D706C6574650000000085
:10B18000456E74657220536C656570206D6F6465E3
:10B19000206E6F772E2E2E0057616B652075702004
:10B1A00066726F6D20736C656570206D6F646500ED
:10B1B00053656E64207061636B6574000102030463
:10B1C000050600000A0D0000307800000406080A99
:10B1D0000E141C006C7063313778785F756172747F
:10B1E0002E6300002020202020202020202020204E
:10B1F000202020203030303030303030303030308F
:10B2000030303030303132333435363738394142EE
:10B210004344454600000000494E4600696E660002
:10B220004E414E006E616E00303132333435363768
:10B23000383961626364656600000000286E756CD1
:10B240006C29000030000000496E66696E697479EF
:10B25000000000004E614E0024000010430000007A
:10B2600098B2000094B2000014B2000014B20000C2
:10B2700014B2000014B2000014B2000014B20000B6
:10B2800014B2000014B2000014B20000FFFFFFFF70
:10B29000FFFFFFFF2E00000049534F2D383835398E
:10B2A0002D31000000000000000000000000F03F11
:10B2B0000000000000002440000000000000594091
:10B2C0000000000000408F40000000000088C340E4
:10B2D00000000000006AF8400000000080842E4159
:10B2E00000000000D01263410000000084D79741A5
:10B2F0000000000065CDCD41000000205FA00242AB
:10B30000000000E876483742000000A2941A6D421F
:10B31000000040E59C30A2420000901EC4BCD64212
:10B3200000003426F56B0C430080E03779C34143BD
:10B3300000A0D8855734764300C84E676DC1AB4333
:10B34000003D9160E458E143408CB5781DAF154451
:10B3500050EFE2D6E41A4B4492D54D06CFF080442C
:10B36000F64AE1C7022DB544B49DD9794378EA4441
:10B3700005000000190000007D0000000000000032
:10B380000080E03779C34143176E05B5B5B89346E1
:10B39000F5F93FE9034F384D321D30F94877825AAD
:10B3A0003CBF737FDD4F1575BC89D897B2D29C3CEA
:10B3B00033A7A8D523F649393DA7F444FD0FA5329C
:10B3C0009D978CCF08BA5B25436FAC642806C80AEA
:10B3D000F8B500BFF8BC08BC9E467047F1000000FD
:10B3E000F8B500BFF8BC08BC9E467047DD00000001
:10B3F0000000000010B4000000000010380500003C
:04B40000802C00009C
:08B40400C84CFF7F01000000AD
:10B4100000000000000000000C1D12E01F100000E2
:10B420000C1D12E01F1000009405001000E1F5054E
:10B4300024000010000000000000000000000000D8
:10B4400000000000000000000000000000000000FC
:10B45000000000005CB200000000000000000000DE
:10B4600000000000000000000000000000000000DC
:10B4700000000000000000000000000000000000CC
:10B4800000000000000000000000000000000000BC
:10B4900000000000000000000000000000000000AC
:10B4A000000000000000000000000000000000009C
:10B4B000000000000000000000000000000000008C
:10B4C000000000000000000000000000000000007C
:10B4D000000000000000000000000000000000006C
:10B4E000000000000000000000000000000000005C
:10B4F000000000000000000000000000000000004C
:10B50000000000000000000000000000000000003B
:10B51000000000000000000000000000000000002B
:10B5200000000000010000004300000000000000D7
:10B5300000000000000000000000000024010010D6
:10B54000240100102C0100102C0100103401001007
:10B55000340100103C0100103C01001044010010B7
:10B56000440100104C0100104C0100105401001067
:10B57000540100105C0100105C0100106401001017
:10B58000640100106C0100106C01001074010010C7
:10B59000740100107C0100107C0100108401001077
:10B5A000840100108C0100108C0100109401001027
:10B5B000940100109C0100109C010010A4010010D7
:10B5C000A4010010AC010010AC010010B401001087
:10B5D000B4010010BC010010BC010010C401001037
:10B5E000C4010010CC010010CC010010D4010010E7
:10B5F000D4010010DC010010DC010010E401001097
:10B60000E4010010EC010010EC010010F401001046
:10B61000F4010010FC010010FC01001004020010F5
:10B62000040200100C0200100C02001014020010A2
:10B63000140200101C0200101C0200102402001052
:10B64000240200102C0200102C0200103402001002
:10B65000340200103C0200103C02001044020010B2
:10B66000440200104C0200104C0200105402001062
:10B67000540200105C0200105C0200106402001012
:10B68000640200106C0200106C02001074020010C2
:10B69000740200107C0200107C0200108402001072
:10B6A000840200108C0200108C0200109402001022
:10B6B000940200109C0200109C020010A4020010D2
:10B6C000A4020010AC020010AC020010B402001082
:10B6D000B4020010BC020010BC020010C402001032
:10B6E000C4020010CC020010CC020010D4020010E2
:10B6F000D4020010DC020010DC020010E402001092
:10B70000E4020010EC020010EC020010F402001041
:10B71000F4020010FC020010FC02001004030010F0
:10B72000040300100C0300100C030010140300109D
:10B73000140300101C0300101C030010240300104D
:10B74000240300102C0300102C03001034030010FD
:10B75000340300103C0300103C03001044030010AD
:10B76000440300104C0300104C030010540300105D
:10B77000540300105C0300105C030010640300100D
:10B78000640300106C0300106C03001074030010BD
:10B79000740300107C0300107C030010840300106D
:10B7A000840300108C0300108C030010940300101D
:10B7B000940300109C0300109C030010A4030010CD
:10B7C000A4030010AC030010AC030010B40300107D
:10B7D000B4030010BC030010BC030010C40300102D
:10B7E000C4030010CC030010CC030010D4030010DD
:10B7F000D4030010DC030010DC030010E40300108D
:10B80000E4030010EC030010EC030010F40300103C
:10B81000F4030010FC030010FC03001004040010EB
:10B82000040400100C0400100C0400101404001098
:10B83000140400101C0400101C0400102404001048
:10B84000240400102C0400102C04001034040010F8
:10B85000340400103C0400103C04001044040010A8
:10B86000440400104C0400104C0400105404001058
:10B87000540400105C0400105C0400106404001008
:10B88000640400106C0400106C04001074040010B8
:10B89000740400107C0400107C0400108404001068
:10B8A000840400108C0400108C0400109404001018
:10B8B000940400109C0400109C040010A4040010C8
:10B8C000A4040010AC040010AC040010B404001078
:10B8D000B4040010BC040010BC040010C404001028
:10B8E000C4040010CC040010CC040010D4040010D8
:10B8F000D4040010DC040010DC040010E404001088
:10B90000E4040010EC040010EC040010F404001037
:10B91000F4040010FC040010FC04001004050010E6
:10B92000040500100C0500100C0500101405001093
:10B93000140500101C0500101C050010FFFFFFFF80
:08B940000000020000000000FD
:00000001FF
